ARM Linker, RVCT4.0 [Build 524] for uVision [Standard]

==============================================================================

Section Cross References

    stm32f10x_adc.o(.text) refers to stm32f10x_rcc.o(.text) for RCC_APB2PeriphResetCmd
    stm32f10x_bkp.o(.text) refers to stm32f10x_rcc.o(.text) for RCC_BackupResetCmd
    stm32f10x_dac.o(.text) refers to stm32f10x_rcc.o(.text) for RCC_APB1PeriphResetCmd
    stm32f10x_gpio.o(.text) refers to stm32f10x_rcc.o(.text) for RCC_APB2PeriphResetCmd
    stm32f10x_pwr.o(.text) refers to stm32f10x_rcc.o(.text) for RCC_APB1PeriphResetCmd
    stm32f10x_rcc.o(.text) refers to stm32f10x_rcc.o(.data) for .data
    main.o(.text) refers to stm32f10x_rcc.o(.text) for RCC_APB2PeriphClockCmd
    main.o(.text) refers to stm32f10x_gpio.o(.text) for GPIO_Init
    main.o(.text) refers to stm32f10x_flash.o(.text) for FLASH_PrefetchBufferCmd
    main.o(.text) refers to qdmx_usb.o(.text) for Set_USBClock
    main.o(.text) refers to usb_init.o(.text) for USB_Init
    main.o(.text) refers to qdmx_adc.o(.text) for m_adc_clk_config
    main.o(.text) refers to usb_regs.o(.text) for GetENDPOINT
    main.o(.text) refers to usb_mem.o(.text) for UserToPMABufferCopy
    main.o(.text) refers to usb_endp.o(.data) for count_in
    stm32f10x_it.o(.text) refers to stm32f10x_adc.o(.text) for ADC_Cmd
    stm32f10x_it.o(.text) refers to usb_regs.o(.text) for SetEPDblBuffCount
    stm32f10x_it.o(.text) refers to qdmx_adc.o(.text) for Control_a
    stm32f10x_it.o(.text) refers to usb_mem.o(.text) for UserToPMABufferCopy
    stm32f10x_it.o(.text) refers to stm32f10x_dma.o(.text) for DMA_ClearFlag
    stm32f10x_it.o(.text) refers to usb_int.o(.text) for CTR_HP
    stm32f10x_it.o(.text) refers to usb_istr.o(.text) for USB_Istr
    stm32f10x_it.o(.text) refers to usb_pwr.o(.data) for bDeviceState
    stm32f10x_it.o(.text) refers to usb_endp.o(.bss) for ADCConvertedValue
    stm32f10x_it.o(.text) refers to stm32f10x_it.o(.data) for Controla_a
    stm32f10x_it.o(.text) refers to usb_endp.o(.data) for count_in
    qdmx_usb.o(.text) refers to stm32f10x_rcc.o(.text) for RCC_APB2PeriphClockCmd
    qdmx_usb.o(.text) refers to stm32f10x_gpio.o(.text) for GPIO_Init
    qdmx_usb.o(.text) refers to misc.o(.text) for NVIC_PriorityGroupConfig
    qdmx_usb.o(.text) refers to usb_pwr.o(.data) for bDeviceState
    qdmx_usb.o(.text) refers to usb_init.o(.bss) for Device_Info
    qdmx_usb.o(.text) refers to usb_desc.o(.data) for Virtual_Com_Port_StringSerial
    usb_endp.o(.text) refers to usb_regs.o(.text) for GetENDPOINT
    usb_endp.o(.text) refers to usb_mem.o(.text) for UserToPMABufferCopy
    usb_endp.o(.text) refers to rt_memclr_w.o(.text) for __aeabi_memclr4
    usb_endp.o(.text) refers to stm32f10x_adc.o(.text) for ADC_Cmd
    usb_endp.o(.text) refers to main.o(.text) for Callback
    usb_endp.o(.text) refers to rand.o(.text) for rand
    usb_endp.o(.text) refers to usb_endp.o(.data) for count_in
    usb_endp.o(.text) refers to usb_endp.o(.bss) for ADCConvertedValue
    usb_endp.o(.text) refers to usb_endp.o(.constdata) for .constdata
    usb_istr.o(.text) refers to usb_int.o(.text) for CTR_LP
    usb_istr.o(.text) refers to usb_istr.o(.data) for wIstr
    usb_istr.o(.text) refers to usb_init.o(.data) for wInterrupt_Mask
    usb_istr.o(.text) refers to usb_prop.o(.data) for Device_Property
    usb_istr.o(.data) refers to usb_endp.o(.text) for EP1_IN_Callback
    usb_istr.o(.data) refers to usb_core.o(.text) for NOP_Process
    usb_prop.o(.text) refers to qdmx_usb.o(.text) for Get_SerialNum
    usb_prop.o(.text) refers to usb_pwr.o(.text) for PowerOn
    usb_prop.o(.text) refers to usb_sil.o(.text) for USB_SIL_Init
    usb_prop.o(.text) refers to usb_regs.o(.text) for SetBTABLE
    usb_prop.o(.text) refers to usb_core.o(.text) for SetDeviceAddress
    usb_prop.o(.text) refers to usb_init.o(.data) for pInformation
    usb_prop.o(.text) refers to usb_pwr.o(.data) for bDeviceState
    usb_prop.o(.text) refers to usb_desc.o(.constdata) for Virtual_Com_Port_ConfigDescriptor
    usb_prop.o(.text) refers to usb_prop.o(.data) for Device_Property
    usb_prop.o(.text) refers to usb_init.o(.bss) for Device_Info
    usb_prop.o(.data) refers to usb_prop.o(.text) for Virtual_Com_Port_init
    usb_prop.o(.data) refers to usb_core.o(.text) for NOP_Process
    usb_prop.o(.data) refers to usb_desc.o(.constdata) for Virtual_Com_Port_DeviceDescriptor
    usb_prop.o(.data) refers to usb_desc.o(.data) for Virtual_Com_Port_StringSerial
    usb_pwr.o(.text) refers to qdmx_usb.o(.text) for USB_Cable_Config
    usb_pwr.o(.text) refers to usb_init.o(.data) for wInterrupt_Mask
    usb_pwr.o(.text) refers to usb_pwr.o(.data) for ResumeS
    qdmx_adc.o(.text) refers to stm32f10x_rcc.o(.text) for RCC_ADCCLKConfig
    qdmx_adc.o(.text) refers to stm32f10x_gpio.o(.text) for GPIO_Init
    qdmx_adc.o(.text) refers to stm32f10x_dma.o(.text) for DMA_DeInit
    qdmx_adc.o(.text) refers to stm32f10x_adc.o(.text) for ADC_Init
    qdmx_adc.o(.text) refers to misc.o(.text) for NVIC_Init
    qdmx_adc.o(.text) refers to usb_endp.o(.bss) for ADCConvertedValue
    qdmx_adc.o(.text) refers to stm32f10x_it.o(.data) for Controla_a
    startup_stm32f10x_md.o(STACK) refers (Special) to heapauxi.o(.text) for __use_two_region_memory
    startup_stm32f10x_md.o(HEAP) refers (Special) to heapauxi.o(.text) for __use_two_region_memory
    startup_stm32f10x_md.o(RESET) refers (Special) to heapauxi.o(.text) for __use_two_region_memory
    startup_stm32f10x_md.o(RESET) refers to startup_stm32f10x_md.o(STACK) for __initial_sp
    startup_stm32f10x_md.o(RESET) refers to startup_stm32f10x_md.o(.text) for Reset_Handler
    startup_stm32f10x_md.o(RESET) refers to stm32f10x_it.o(.text) for NMI_Handler
    startup_stm32f10x_md.o(.text) refers (Special) to heapauxi.o(.text) for __use_two_region_memory
    startup_stm32f10x_md.o(.text) refers to __main.o(!!!main) for __main
    startup_stm32f10x_md.o(.text) refers to startup_stm32f10x_md.o(HEAP) for Heap_Mem
    startup_stm32f10x_md.o(.text) refers to startup_stm32f10x_md.o(STACK) for Stack_Mem
    usb_core.o(.text) refers to usb_regs.o(.text) for ClearDTOG_TX
    usb_core.o(.text) refers to usb_init.o(.data) for pInformation
    usb_core.o(.text) refers to usb_prop.o(.data) for Device_Table
    usb_core.o(.text) refers to usb_core.o(.data) for StatusInfo
    usb_core.o(.text) refers to usb_mem.o(.text) for PMAToUserBufferCopy
    usb_core.o(.text) refers to usb_int.o(.data) for SaveRState
    usb_init.o(.text) refers to usb_init.o(.bss) for Device_Info
    usb_init.o(.text) refers to usb_init.o(.data) for pInformation
    usb_init.o(.text) refers to usb_prop.o(.data) for Device_Property
    usb_int.o(.text) refers to usb_core.o(.text) for In0_Process
    usb_int.o(.text) refers to usb_istr.o(.data) for wIstr
    usb_int.o(.text) refers to usb_init.o(.data) for EPindex
    usb_int.o(.text) refers to usb_int.o(.data) for SaveRState
    usb_sil.o(.text) refers to usb_regs.o(.text) for GetEPTxAddr
    usb_sil.o(.text) refers to usb_mem.o(.text) for UserToPMABufferCopy
    usb_sil.o(.text) refers to usb_init.o(.data) for wInterrupt_Mask
    rand.o(.text) refers (Special) to libinit2.o(.ARM.Collect$$libinit$$00000009) for __rt_lib_init_rand_2
    rand.o(.text) refers to rand.o(.data) for .data
    rand.o(.text) refers to rand.o(.bss) for .bss
    rand.o(.bss) refers (Special) to libinit2.o(.ARM.Collect$$libinit$$00000009) for __rt_lib_init_rand_2
    rand.o(.data) refers (Special) to libinit2.o(.ARM.Collect$$libinit$$00000009) for __rt_lib_init_rand_2
    __main.o(!!!main) refers to rtentry.o(.ARM.Collect$$rtentry$$00000000) for __rt_entry
    rtentry.o(.ARM.Collect$$rtentry$$00000000) refers (Special) to rtentry2.o(.ARM.Collect$$rtentry$$0000000A) for __rt_entry_li
    rtentry.o(.ARM.Collect$$rtentry$$00000000) refers (Special) to rtentry2.o(.ARM.Collect$$rtentry$$0000000D) for __rt_entry_main
    rtentry.o(.ARM.Collect$$rtentry$$00000000) refers (Special) to rtentry2.o(.ARM.Collect$$rtentry$$0000000C) for __rt_entry_postli_1
    rtentry.o(.ARM.Collect$$rtentry$$00000000) refers (Special) to rtentry2.o(.ARM.Collect$$rtentry$$00000009) for __rt_entry_postsh_1
    rtentry.o(.ARM.Collect$$rtentry$$00000000) refers (Special) to rtentry2.o(.ARM.Collect$$rtentry$$00000002) for __rt_entry_presh_1
    rtentry.o(.ARM.Collect$$rtentry$$00000000) refers (Special) to rtentry4.o(.ARM.Collect$$rtentry$$00000004) for __rt_entry_sh
    rtentry.o(.ARM.exidx) refers (Special) to rtentry2.o(.ARM.Collect$$rtentry$$0000000A) for __rt_entry_li
    rtentry.o(.ARM.exidx) refers (Special) to rtentry2.o(.ARM.Collect$$rtentry$$0000000D) for __rt_entry_main
    rtentry.o(.ARM.exidx) refers (Special) to rtentry2.o(.ARM.Collect$$rtentry$$0000000C) for __rt_entry_postli_1
    rtentry.o(.ARM.exidx) refers (Special) to rtentry2.o(.ARM.Collect$$rtentry$$00000009) for __rt_entry_postsh_1
    rtentry.o(.ARM.exidx) refers (Special) to rtentry2.o(.ARM.Collect$$rtentry$$00000002) for __rt_entry_presh_1
    rtentry.o(.ARM.exidx) refers (Special) to rtentry4.o(.ARM.Collect$$rtentry$$00000004) for __rt_entry_sh
    rtentry.o(.ARM.exidx) refers to rtentry.o(.ARM.Collect$$rtentry$$00000000) for .ARM.Collect$$rtentry$$00000000
    libinit2.o(.ARM.Collect$$libinit$$00000009) refers (Weak) to rand.o(.text) for _rand_init
    libinit2.o(.ARM.Collect$$libinit$$0000000C) refers to libinit2.o(.ARM.Collect$$libinit$$0000000B) for .ARM.Collect$$libinit$$0000000B
    libinit2.o(.ARM.Collect$$libinit$$0000000E) refers to libinit2.o(.ARM.Collect$$libinit$$0000000B) for .ARM.Collect$$libinit$$0000000B
    libinit2.o(.ARM.Collect$$libinit$$00000010) refers to libinit2.o(.ARM.Collect$$libinit$$0000000B) for .ARM.Collect$$libinit$$0000000B
    libinit2.o(.ARM.Collect$$libinit$$00000012) refers to libinit2.o(.ARM.Collect$$libinit$$0000000B) for .ARM.Collect$$libinit$$0000000B
    libinit2.o(.ARM.Collect$$libinit$$00000014) refers to libinit2.o(.ARM.Collect$$libinit$$0000000B) for .ARM.Collect$$libinit$$0000000B
    libinit2.o(.ARM.Collect$$libinit$$00000022) refers to argv_veneer.o(.emb_text) for __ARM_argv_veneer
    libinit2.o(.ARM.Collect$$libinit$$00000023) refers to argv_veneer.o(.emb_text) for __ARM_argv_veneer
    rtentry2.o(.ARM.Collect$$rtentry$$00000008) refers to boardinit2.o(.text) for _platform_post_stackheap_init
    rtentry2.o(.ARM.Collect$$rtentry$$0000000A) refers to libinit.o(.ARM.Collect$$libinit$$00000000) for __rt_lib_init
    rtentry2.o(.ARM.Collect$$rtentry$$0000000B) refers to boardinit3.o(.text) for _platform_post_lib_init
    rtentry2.o(.ARM.Collect$$rtentry$$0000000D) refers to main.o(.text) for main
    rtentry2.o(.ARM.Collect$$rtentry$$0000000D) refers to exit.o(.text) for exit
    rtentry2.o(.ARM.exidx) refers to rtentry2.o(.ARM.Collect$$rtentry$$00000001) for .ARM.Collect$$rtentry$$00000001
    rtentry2.o(.ARM.exidx) refers to rtentry2.o(.ARM.Collect$$rtentry$$00000002) for .ARM.Collect$$rtentry$$00000002
    rtentry2.o(.ARM.exidx) refers to rtentry2.o(.ARM.Collect$$rtentry$$00000008) for .ARM.Collect$$rtentry$$00000008
    rtentry2.o(.ARM.exidx) refers to rtentry2.o(.ARM.Collect$$rtentry$$00000009) for .ARM.Collect$$rtentry$$00000009
    rtentry2.o(.ARM.exidx) refers to rtentry2.o(.ARM.Collect$$rtentry$$0000000A) for .ARM.Collect$$rtentry$$0000000A
    rtentry2.o(.ARM.exidx) refers to rtentry2.o(.ARM.Collect$$rtentry$$0000000B) for .ARM.Collect$$rtentry$$0000000B
    rtentry2.o(.ARM.exidx) refers to rtentry2.o(.ARM.Collect$$rtentry$$0000000C) for .ARM.Collect$$rtentry$$0000000C
    rtentry2.o(.ARM.exidx) refers to rtentry2.o(.ARM.Collect$$rtentry$$0000000D) for .ARM.Collect$$rtentry$$0000000D
    rtentry4.o(.ARM.Collect$$rtentry$$00000004) refers to sys_stackheap_outer.o(.text) for __user_setup_stackheap
    rtentry4.o(.ARM.exidx) refers to rtentry4.o(.ARM.Collect$$rtentry$$00000004) for .ARM.Collect$$rtentry$$00000004
    argv_veneer.o(.emb_text) refers to no_argv.o(.text) for __ARM_get_argv
    sys_stackheap_outer.o(.text) refers to libspace.o(.text) for __user_perproc_libspace
    sys_stackheap_outer.o(.text) refers to startup_stm32f10x_md.o(.text) for __user_initial_stackheap
    exit.o(.text) refers to rtexit.o(.ARM.Collect$$rtexit$$00000000) for __rt_exit
    _get_argv_nomalloc.o(.text) refers (Special) to hrguard.o(.text) for __heap_region$guard
    _get_argv_nomalloc.o(.text) refers to defsig_rtmem_outer.o(.text) for __rt_SIGRTMEM
    _get_argv_nomalloc.o(.text) refers to sys_command.o(.text) for _sys_command_string
    libinit.o(.ARM.Collect$$libinit$$00000000) refers (Special) to libinit2.o(.ARM.Collect$$libinit$$0000002A) for __rt_lib_init_alloca_1
    libinit.o(.ARM.Collect$$libinit$$00000000) refers (Special) to libinit2.o(.ARM.Collect$$libinit$$00000028) for __rt_lib_init_argv_1
    libinit.o(.ARM.Collect$$libinit$$00000000) refers (Special) to libinit2.o(.ARM.Collect$$libinit$$00000017) for __rt_lib_init_atexit_1
    libinit.o(.ARM.Collect$$libinit$$00000000) refers (Special) to libinit2.o(.ARM.Collect$$libinit$$0000001D) for __rt_lib_init_clock_1
    libinit.o(.ARM.Collect$$libinit$$00000000) refers (Special) to libinit2.o(.ARM.Collect$$libinit$$0000002E) for __rt_lib_init_cpp_1
    libinit.o(.ARM.Collect$$libinit$$00000000) refers (Special) to libinit2.o(.ARM.Collect$$libinit$$0000002C) for __rt_lib_init_exceptions_1
    libinit.o(.ARM.Collect$$libinit$$00000000) refers (Special) to libinit2.o(.ARM.Collect$$libinit$$0000001B) for __rt_lib_init_fp_trap_1
    libinit.o(.ARM.Collect$$libinit$$00000000) refers (Special) to libinit2.o(.ARM.Collect$$libinit$$0000001F) for __rt_lib_init_getenv_1
    libinit.o(.ARM.Collect$$libinit$$00000000) refers (Special) to libinit2.o(.ARM.Collect$$libinit$$00000006) for __rt_lib_init_heap_1
    libinit.o(.ARM.Collect$$libinit$$00000000) refers (Special) to libinit2.o(.ARM.Collect$$libinit$$0000000D) for __rt_lib_init_lc_collate_1
    libinit.o(.ARM.Collect$$libinit$$00000000) refers (Special) to libinit2.o(.ARM.Collect$$libinit$$0000000F) for __rt_lib_init_lc_ctype_1
    libinit.o(.ARM.Collect$$libinit$$00000000) refers (Special) to libinit2.o(.ARM.Collect$$libinit$$00000011) for __rt_lib_init_lc_monetary_1
    libinit.o(.ARM.Collect$$libinit$$00000000) refers (Special) to libinit2.o(.ARM.Collect$$libinit$$00000013) for __rt_lib_init_lc_numeric_1
    libinit.o(.ARM.Collect$$libinit$$00000000) refers (Special) to libinit2.o(.ARM.Collect$$libinit$$00000015) for __rt_lib_init_lc_time_1
    libinit.o(.ARM.Collect$$libinit$$00000000) refers (Special) to libinit2.o(.ARM.Collect$$libinit$$0000000A) for __rt_lib_init_rand_1
    libinit.o(.ARM.Collect$$libinit$$00000000) refers (Special) to libinit2.o(.ARM.Collect$$libinit$$0000002F) for __rt_lib_init_return
    libinit.o(.ARM.Collect$$libinit$$00000000) refers (Special) to libinit2.o(.ARM.Collect$$libinit$$00000019) for __rt_lib_init_signal_1
    libinit.o(.ARM.Collect$$libinit$$00000000) refers (Special) to libinit2.o(.ARM.Collect$$libinit$$00000021) for __rt_lib_init_stdio_1
    libinit.o(.ARM.Collect$$libinit$$00000000) refers (Special) to libinit2.o(.ARM.Collect$$libinit$$00000008) for __rt_lib_init_user_alloc_1
    sys_command.o(.text) refers (Special) to use_no_semi.o(.text) for __I$use$semihosting
    libspace.o(.text) refers to libspace.o(.bss) for __libspace_start
    rtexit.o(.ARM.Collect$$rtexit$$00000000) refers (Special) to rtexit2.o(.ARM.Collect$$rtexit$$00000004) for __rt_exit_exit
    rtexit.o(.ARM.Collect$$rtexit$$00000000) refers (Special) to rtexit2.o(.ARM.Collect$$rtexit$$00000003) for __rt_exit_ls
    rtexit.o(.ARM.Collect$$rtexit$$00000000) refers (Special) to rtexit2.o(.ARM.Collect$$rtexit$$00000002) for __rt_exit_prels_1
    rtexit.o(.ARM.exidx) refers (Special) to rtexit2.o(.ARM.Collect$$rtexit$$00000004) for __rt_exit_exit
    rtexit.o(.ARM.exidx) refers (Special) to rtexit2.o(.ARM.Collect$$rtexit$$00000003) for __rt_exit_ls
    rtexit.o(.ARM.exidx) refers (Special) to rtexit2.o(.ARM.Collect$$rtexit$$00000002) for __rt_exit_prels_1
    rtexit.o(.ARM.exidx) refers to rtexit.o(.ARM.Collect$$rtexit$$00000000) for .ARM.Collect$$rtexit$$00000000
    defsig_rtmem_outer.o(.text) refers to defsig_rtmem_inner.o(.text) for __rt_SIGRTMEM_inner
    defsig_rtmem_outer.o(.text) refers to defsig_exit.o(.text) for __sig_exit
    defsig_rtmem_formal.o(.text) refers to rt_raise.o(.text) for __rt_raise
    rtexit2.o(.ARM.Collect$$rtexit$$00000003) refers to libshutdown.o(.ARM.Collect$$libshutdown$$00000000) for __rt_lib_shutdown
    rtexit2.o(.ARM.Collect$$rtexit$$00000004) refers to sys_exit.o(.text) for _sys_exit
    rtexit2.o(.ARM.exidx) refers to rtexit2.o(.ARM.Collect$$rtexit$$00000001) for .ARM.Collect$$rtexit$$00000001
    rtexit2.o(.ARM.exidx) refers to rtexit2.o(.ARM.Collect$$rtexit$$00000002) for .ARM.Collect$$rtexit$$00000002
    rtexit2.o(.ARM.exidx) refers to rtexit2.o(.ARM.Collect$$rtexit$$00000003) for .ARM.Collect$$rtexit$$00000003
    rtexit2.o(.ARM.exidx) refers to rtexit2.o(.ARM.Collect$$rtexit$$00000004) for .ARM.Collect$$rtexit$$00000004
    rt_raise.o(.text) refers to __raise.o(.text) for __raise
    rt_raise.o(.text) refers to sys_exit.o(.text) for _sys_exit
    defsig_exit.o(.text) refers to sys_exit.o(.text) for _sys_exit
    defsig_rtmem_inner.o(.text) refers to defsig_general.o(.text) for __default_signal_display
    sys_exit.o(.text) refers to use_no_semi.o(.text) for __I$use$semihosting
    __raise.o(.text) refers to defsig.o(CL$$defsig) for __default_signal_handler
    defsig_general.o(.text) refers to sys_wrch.o(.text) for _ttywrch
    libshutdown.o(.ARM.Collect$$libshutdown$$00000000) refers (Special) to libshutdown2.o(.ARM.Collect$$libshutdown$$00000006) for __rt_lib_shutdown_fp_trap_1
    libshutdown.o(.ARM.Collect$$libshutdown$$00000000) refers (Special) to libshutdown2.o(.ARM.Collect$$libshutdown$$0000000E) for __rt_lib_shutdown_heap_1
    libshutdown.o(.ARM.Collect$$libshutdown$$00000000) refers (Special) to libshutdown2.o(.ARM.Collect$$libshutdown$$0000000F) for __rt_lib_shutdown_return
    libshutdown.o(.ARM.Collect$$libshutdown$$00000000) refers (Special) to libshutdown2.o(.ARM.Collect$$libshutdown$$00000009) for __rt_lib_shutdown_signal_1
    libshutdown.o(.ARM.Collect$$libshutdown$$00000000) refers (Special) to libshutdown2.o(.ARM.Collect$$libshutdown$$00000003) for __rt_lib_shutdown_stdio_1
    libshutdown.o(.ARM.Collect$$libshutdown$$00000000) refers (Special) to libshutdown2.o(.ARM.Collect$$libshutdown$$0000000B) for __rt_lib_shutdown_user_alloc_1
    sys_wrch.o(.text) refers (Special) to use_no_semi.o(.text) for __I$use$semihosting
    defsig.o(CL$$defsig) refers to defsig_rtmem_inner.o(.text) for __rt_SIGRTMEM_inner
    defsig_abrt_inner.o(.text) refers to defsig_general.o(.text) for __default_signal_display
    defsig_fpe_inner.o(.text) refers to defsig_general.o(.text) for __default_signal_display
    defsig_rtred_inner.o(.text) refers to defsig_general.o(.text) for __default_signal_display
    defsig_stak_inner.o(.text) refers to defsig_general.o(.text) for __default_signal_display
    defsig_pvfn_inner.o(.text) refers to defsig_general.o(.text) for __default_signal_display
    defsig_cppl_inner.o(.text) refers to defsig_general.o(.text) for __default_signal_display
    defsig_segv_inner.o(.text) refers to defsig_general.o(.text) for __default_signal_display
    defsig_other.o(.text) refers to defsig_general.o(.text) for __default_signal_display


==============================================================================

Removing Unused input sections from the image.

    Removing stm32f10x_bkp.o(.text), (172 bytes).
    Removing stm32f10x_crc.o(.text), (72 bytes).
    Removing stm32f10x_dac.o(.text), (356 bytes).
    Removing stm32f10x_dbgmcu.o(.text), (48 bytes).
    Removing stm32f10x_exti.o(.text), (336 bytes).
    Removing stm32f10x_fsmc.o(.text), (1536 bytes).
    Removing stm32f10x_iwdg.o(.text), (64 bytes).
    Removing stm32f10x_pwr.o(.text), (196 bytes).
    Removing core_cm3.o(.emb_text), (32 bytes).
    Removing system_stm32f10x.o(.text), (292 bytes).
    Removing system_stm32f10x.o(.constdata), (20 bytes).

11 unused section(s) (total 3124 bytes) removed from the image.

==============================================================================

Image Symbol Table

    Local Symbols

    Symbol Name                              Value     Ov Type        Size  Object(Section)

    ../../angel/boardlib.s                   0x00000000   Number         0  boardshut.o ABSOLUTE
    ../../angel/boardlib.s                   0x00000000   Number         0  boardinit1.o ABSOLUTE
    ../../angel/boardlib.s                   0x00000000   Number         0  boardinit2.o ABSOLUTE
    ../../angel/boardlib.s                   0x00000000   Number         0  boardinit3.o ABSOLUTE
    ../../angel/dczerorl2.s                  0x00000000   Number         0  __dczerorl2.o ABSOLUTE
    ../../angel/handlers.s                   0x00000000   Number         0  __scatter_zi.o ABSOLUTE
    ../../angel/kernel.s                     0x00000000   Number         0  rtentry.o ABSOLUTE
    ../../angel/kernel.s                     0x00000000   Number         0  rtentry2.o ABSOLUTE
    ../../angel/kernel.s                     0x00000000   Number         0  rtentry4.o ABSOLUTE
    ../../angel/kernel.s                     0x00000000   Number         0  rtexit.o ABSOLUTE
    ../../angel/kernel.s                     0x00000000   Number         0  rtexit2.o ABSOLUTE
    ../../angel/rt.s                         0x00000000   Number         0  rt_raise.o ABSOLUTE
    ../../angel/scatter.s                    0x00000000   Number         0  __scatter.o ABSOLUTE
    ../../angel/startup.s                    0x00000000   Number         0  __main.o ABSOLUTE
    ../../angel/sys.s                        0x00000000   Number         0  sys_stackheap_outer.o ABSOLUTE
    ../../angel/sys.s                        0x00000000   Number         0  libspace.o ABSOLUTE
    ../../angel/sys.s                        0x00000000   Number         0  sys_exit.o ABSOLUTE
    ../../angel/sys.s                        0x00000000   Number         0  use_no_semi.o ABSOLUTE
    ../../angel/sysapp.c                     0x00000000   Number         0  sys_wrch.o ABSOLUTE
    ../../angel/sysapp.c                     0x00000000   Number         0  sys_command.o ABSOLUTE
    ../../armsys.c                           0x00000000   Number         0  _get_argv_nomalloc.o ABSOLUTE
    ../../armsys.c                           0x00000000   Number         0  no_argv.o ABSOLUTE
    ../../armsys.c                           0x00000000   Number         0  argv_veneer.o ABSOLUTE
    ../../armsys.c                           0x00000000   Number         0  argv_veneer.o ABSOLUTE
    ../../fpinit.s                           0x00000000   Number         0  fpinit.o ABSOLUTE
    ../../heapalloc.c                        0x00000000   Number         0  hrguard.o ABSOLUTE
    ../../heapaux.c                          0x00000000   Number         0  heapauxi.o ABSOLUTE
    ../../libinit.s                          0x00000000   Number         0  libshutdown2.o ABSOLUTE
    ../../libinit.s                          0x00000000   Number         0  libinit2.o ABSOLUTE
    ../../libinit.s                          0x00000000   Number         0  libshutdown.o ABSOLUTE
    ../../libinit.s                          0x00000000   Number         0  libinit.o ABSOLUTE
    ../../memcpset.s                         0x00000000   Number         0  rt_memclr_w.o ABSOLUTE
    ../../signal.c                           0x00000000   Number         0  defsig_rtmem_inner.o ABSOLUTE
    ../../signal.c                           0x00000000   Number         0  defsig_exit.o ABSOLUTE
    ../../signal.c                           0x00000000   Number         0  defsig_rtmem_formal.o ABSOLUTE
    ../../signal.c                           0x00000000   Number         0  defsig_general.o ABSOLUTE
    ../../signal.c                           0x00000000   Number         0  defsig_rtmem_outer.o ABSOLUTE
    ../../signal.c                           0x00000000   Number         0  defsig_abrt_inner.o ABSOLUTE
    ../../signal.c                           0x00000000   Number         0  defsig_fpe_inner.o ABSOLUTE
    ../../signal.c                           0x00000000   Number         0  defsig_rtred_inner.o ABSOLUTE
    ../../signal.c                           0x00000000   Number         0  defsig_stak_inner.o ABSOLUTE
    ../../signal.c                           0x00000000   Number         0  defsig_pvfn_inner.o ABSOLUTE
    ../../signal.c                           0x00000000   Number         0  defsig_cppl_inner.o ABSOLUTE
    ../../signal.c                           0x00000000   Number         0  defsig_segv_inner.o ABSOLUTE
    ../../signal.c                           0x00000000   Number         0  defsig_other.o ABSOLUTE
    ../../signal.c                           0x00000000   Number         0  __raise.o ABSOLUTE
    ../../signal.s                           0x00000000   Number         0  defsig.o ABSOLUTE
    ../../stdlib.c                           0x00000000   Number         0  exit.o ABSOLUTE
    ../../stdlib.c                           0x00000000   Number         0  rand.o ABSOLUTE
    ..\CM3\core_cm3.c                        0x00000000   Number         0  core_cm3.o ABSOLUTE
    ..\CM3\startup\arm\startup_stm32f10x_md.s 0x00000000   Number         0  startup_stm32f10x_md.o ABSOLUTE
    ..\CM3\system_stm32f10x.c                0x00000000   Number         0  system_stm32f10x.o ABSOLUTE
    ..\STM32F10x_StdPeriph_Driver\src\misc.c 0x00000000   Number         0  misc.o ABSOLUTE
    ..\STM32F10x_StdPeriph_Driver\src\stm32f10x_adc.c 0x00000000   Number         0  stm32f10x_adc.o ABSOLUTE
    ..\STM32F10x_StdPeriph_Driver\src\stm32f10x_bkp.c 0x00000000   Number         0  stm32f10x_bkp.o ABSOLUTE
    ..\STM32F10x_StdPeriph_Driver\src\stm32f10x_crc.c 0x00000000   Number         0  stm32f10x_crc.o ABSOLUTE
    ..\STM32F10x_StdPeriph_Driver\src\stm32f10x_dac.c 0x00000000   Number         0  stm32f10x_dac.o ABSOLUTE
    ..\STM32F10x_StdPeriph_Driver\src\stm32f10x_dbgmcu.c 0x00000000   Number         0  stm32f10x_dbgmcu.o ABSOLUTE
    ..\STM32F10x_StdPeriph_Driver\src\stm32f10x_dma.c 0x00000000   Number         0  stm32f10x_dma.o ABSOLUTE
    ..\STM32F10x_StdPeriph_Driver\src\stm32f10x_exti.c 0x00000000   Number         0  stm32f10x_exti.o ABSOLUTE
    ..\STM32F10x_StdPeriph_Driver\src\stm32f10x_flash.c 0x00000000   Number         0  stm32f10x_flash.o ABSOLUTE
    ..\STM32F10x_StdPeriph_Driver\src\stm32f10x_fsmc.c 0x00000000   Number         0  stm32f10x_fsmc.o ABSOLUTE
    ..\STM32F10x_StdPeriph_Driver\src\stm32f10x_gpio.c 0x00000000   Number         0  stm32f10x_gpio.o ABSOLUTE
    ..\STM32F10x_StdPeriph_Driver\src\stm32f10x_iwdg.c 0x00000000   Number         0  stm32f10x_iwdg.o ABSOLUTE
    ..\STM32F10x_StdPeriph_Driver\src\stm32f10x_pwr.c 0x00000000   Number         0  stm32f10x_pwr.o ABSOLUTE
    ..\STM32F10x_StdPeriph_Driver\src\stm32f10x_rcc.c 0x00000000   Number         0  stm32f10x_rcc.o ABSOLUTE
    ..\STM32_USB-FS-Device_Driver\src\usb_core.c 0x00000000   Number         0  usb_core.o ABSOLUTE
    ..\STM32_USB-FS-Device_Driver\src\usb_init.c 0x00000000   Number         0  usb_init.o ABSOLUTE
    ..\STM32_USB-FS-Device_Driver\src\usb_int.c 0x00000000   Number         0  usb_int.o ABSOLUTE
    ..\STM32_USB-FS-Device_Driver\src\usb_mem.c 0x00000000   Number         0  usb_mem.o ABSOLUTE
    ..\STM32_USB-FS-Device_Driver\src\usb_regs.c 0x00000000   Number         0  usb_regs.o ABSOLUTE
    ..\STM32_USB-FS-Device_Driver\src\usb_sil.c 0x00000000   Number         0  usb_sil.o ABSOLUTE
    ..\\CM3\\core_cm3.c                      0x00000000   Number         0  core_cm3.o ABSOLUTE
    ..\user\main.c                           0x00000000   Number         0  main.o ABSOLUTE
    ..\user\qdmx_adc.c                       0x00000000   Number         0  qdmx_adc.o ABSOLUTE
    ..\user\qdmx_usb.c                       0x00000000   Number         0  qdmx_usb.o ABSOLUTE
    ..\user\stm32f10x_it.c                   0x00000000   Number         0  stm32f10x_it.o ABSOLUTE
    ..\user\usb_desc.c                       0x00000000   Number         0  usb_desc.o ABSOLUTE
    ..\user\usb_endp.c                       0x00000000   Number         0  usb_endp.o ABSOLUTE
    ..\user\usb_istr.c                       0x00000000   Number         0  usb_istr.o ABSOLUTE
    ..\user\usb_prop.c                       0x00000000   Number         0  usb_prop.o ABSOLUTE
    ..\user\usb_pwr.c                        0x00000000   Number         0  usb_pwr.o ABSOLUTE
    dc.s                                     0x00000000   Number         0  dc.o ABSOLUTE
    RESET                                    0x08000000   Section      236  startup_stm32f10x_md.o(RESET)
    !!!main                                  0x080000ec   Section        8  __main.o(!!!main)
    !!!scatter                               0x080000f4   Section       52  __scatter.o(!!!scatter)
    !!dczerorl2                              0x08000128   Section       90  __dczerorl2.o(!!dczerorl2)
    !!handler_zi                             0x08000184   Section       28  __scatter_zi.o(!!handler_zi)
    .ARM.Collect$$libinit$$00000000          0x080001a0   Section        6  libinit.o(.ARM.Collect$$libinit$$00000000)
    .ARM.Collect$$libinit$$00000006          0x080001a6   Section        0  libinit2.o(.ARM.Collect$$libinit$$00000006)
    .ARM.Collect$$libinit$$00000008          0x080001a6   Section        0  libinit2.o(.ARM.Collect$$libinit$$00000008)
    .ARM.Collect$$libinit$$00000009          0x080001a6   Section        4  libinit2.o(.ARM.Collect$$libinit$$00000009)
    .ARM.Collect$$libinit$$0000000A          0x080001aa   Section        0  libinit2.o(.ARM.Collect$$libinit$$0000000A)
    .ARM.Collect$$libinit$$0000000D          0x080001aa   Section        0  libinit2.o(.ARM.Collect$$libinit$$0000000D)
    .ARM.Collect$$libinit$$0000000F          0x080001aa   Section        0  libinit2.o(.ARM.Collect$$libinit$$0000000F)
    .ARM.Collect$$libinit$$00000011          0x080001aa   Section        0  libinit2.o(.ARM.Collect$$libinit$$00000011)
    .ARM.Collect$$libinit$$00000013          0x080001aa   Section        0  libinit2.o(.ARM.Collect$$libinit$$00000013)
    .ARM.Collect$$libinit$$00000015          0x080001aa   Section        0  libinit2.o(.ARM.Collect$$libinit$$00000015)
    .ARM.Collect$$libinit$$00000017          0x080001aa   Section        0  libinit2.o(.ARM.Collect$$libinit$$00000017)
    .ARM.Collect$$libinit$$00000019          0x080001aa   Section        0  libinit2.o(.ARM.Collect$$libinit$$00000019)
    .ARM.Collect$$libinit$$0000001B          0x080001aa   Section        0  libinit2.o(.ARM.Collect$$libinit$$0000001B)
    .ARM.Collect$$libinit$$0000001D          0x080001aa   Section        0  libinit2.o(.ARM.Collect$$libinit$$0000001D)
    .ARM.Collect$$libinit$$0000001F          0x080001aa   Section        0  libinit2.o(.ARM.Collect$$libinit$$0000001F)
    .ARM.Collect$$libinit$$00000021          0x080001aa   Section        0  libinit2.o(.ARM.Collect$$libinit$$00000021)
    .ARM.Collect$$libinit$$00000028          0x080001aa   Section        0  libinit2.o(.ARM.Collect$$libinit$$00000028)
    .ARM.Collect$$libinit$$0000002A          0x080001aa   Section        0  libinit2.o(.ARM.Collect$$libinit$$0000002A)
    .ARM.Collect$$libinit$$0000002C          0x080001aa   Section        0  libinit2.o(.ARM.Collect$$libinit$$0000002C)
    .ARM.Collect$$libinit$$0000002E          0x080001aa   Section        0  libinit2.o(.ARM.Collect$$libinit$$0000002E)
    .ARM.Collect$$libinit$$0000002F          0x080001aa   Section        2  libinit2.o(.ARM.Collect$$libinit$$0000002F)
    .ARM.Collect$$libshutdown$$00000000      0x080001ac   Section        2  libshutdown.o(.ARM.Collect$$libshutdown$$00000000)
    .ARM.Collect$$libshutdown$$00000003      0x080001ae   Section        0  libshutdown2.o(.ARM.Collect$$libshutdown$$00000003)
    .ARM.Collect$$libshutdown$$00000006      0x080001ae   Section        0  libshutdown2.o(.ARM.Collect$$libshutdown$$00000006)
    .ARM.Collect$$libshutdown$$00000009      0x080001ae   Section        0  libshutdown2.o(.ARM.Collect$$libshutdown$$00000009)
    .ARM.Collect$$libshutdown$$0000000B      0x080001ae   Section        0  libshutdown2.o(.ARM.Collect$$libshutdown$$0000000B)
    .ARM.Collect$$libshutdown$$0000000E      0x080001ae   Section        0  libshutdown2.o(.ARM.Collect$$libshutdown$$0000000E)
    .ARM.Collect$$libshutdown$$0000000F      0x080001ae   Section        2  libshutdown2.o(.ARM.Collect$$libshutdown$$0000000F)
    .ARM.Collect$$rtentry$$00000000          0x080001b0   Section        0  rtentry.o(.ARM.Collect$$rtentry$$00000000)
    .ARM.Collect$$rtentry$$00000002          0x080001b0   Section        0  rtentry2.o(.ARM.Collect$$rtentry$$00000002)
    .ARM.Collect$$rtentry$$00000004          0x080001b0   Section        6  rtentry4.o(.ARM.Collect$$rtentry$$00000004)
    .ARM.Collect$$rtentry$$00000009          0x080001b6   Section        0  rtentry2.o(.ARM.Collect$$rtentry$$00000009)
    .ARM.Collect$$rtentry$$0000000A          0x080001b6   Section        4  rtentry2.o(.ARM.Collect$$rtentry$$0000000A)
    .ARM.Collect$$rtentry$$0000000C          0x080001ba   Section        0  rtentry2.o(.ARM.Collect$$rtentry$$0000000C)
    .ARM.Collect$$rtentry$$0000000D          0x080001ba   Section        8  rtentry2.o(.ARM.Collect$$rtentry$$0000000D)
    .ARM.Collect$$rtexit$$00000000           0x080001c2   Section        0  rtexit.o(.ARM.Collect$$rtexit$$00000000)
    .ARM.Collect$$rtexit$$00000002           0x080001c2   Section        0  rtexit2.o(.ARM.Collect$$rtexit$$00000002)
    .ARM.Collect$$rtexit$$00000003           0x080001c2   Section        4  rtexit2.o(.ARM.Collect$$rtexit$$00000003)
    .ARM.Collect$$rtexit$$00000004           0x080001c6   Section        4  rtexit2.o(.ARM.Collect$$rtexit$$00000004)
    .text                                    0x080001cc   Section      224  misc.o(.text)
    .text                                    0x080002ac   Section     1058  stm32f10x_adc.o(.text)
    .text                                    0x080006d0   Section      592  stm32f10x_dma.o(.text)
    .text                                    0x08000920   Section     1320  stm32f10x_flash.o(.text)
    delay                                    0x080009a9   Thumb Code    14  stm32f10x_flash.o(.text)
    .text                                    0x08000e48   Section      796  stm32f10x_gpio.o(.text)
    .text                                    0x08001164   Section      908  stm32f10x_rcc.o(.text)
    .text                                    0x080014f0   Section      392  main.o(.text)
    .text                                    0x08001678   Section      584  stm32f10x_it.o(.text)
    .text                                    0x080018c0   Section      248  qdmx_usb.o(.text)
    .text                                    0x080019b8   Section     1288  usb_endp.o(.text)
    .text                                    0x08001ec0   Section      140  usb_istr.o(.text)
    .text                                    0x08001f4c   Section      608  usb_prop.o(.text)
    .text                                    0x080021ac   Section      352  usb_pwr.o(.text)
    .text                                    0x0800230c   Section     1356  qdmx_adc.o(.text)
    .text                                    0x08002858   Section       52  startup_stm32f10x_md.o(.text)
    .text                                    0x0800288c   Section     2904  usb_core.o(.text)
    DataStageOut                             0x08002ccf   Thumb Code   166  usb_core.o(.text)
    DataStageIn                              0x08002d75   Thumb Code   166  usb_core.o(.text)
    NoData_Setup0                            0x08002e1b   Thumb Code   300  usb_core.o(.text)
    Data_Setup0                              0x08002f47   Thumb Code   670  usb_core.o(.text)
    .text                                    0x080033e4   Section       60  usb_init.o(.text)
    .text                                    0x08003420   Section      820  usb_int.o(.text)
    .text                                    0x08003754   Section       88  usb_mem.o(.text)
    .text                                    0x080037ac   Section     2088  usb_regs.o(.text)
    .text                                    0x08003fd4   Section      132  usb_sil.o(.text)
    .text                                    0x08004058   Section      120  rand.o(.text)
    .text                                    0x080040d0   Section       78  rt_memclr_w.o(.text)
    .text                                    0x0800411e   Section        6  heapauxi.o(.text)
    .text                                    0x08004124   Section       74  sys_stackheap_outer.o(.text)
    .text                                    0x0800416e   Section       12  exit.o(.text)
    .text                                    0x0800417c   Section        8  libspace.o(.text)
    .text                                    0x08004184   Section        2  use_no_semi.o(.text)
    .text                                    0x08004188   Section       20  sys_exit.o(.text)
    .constdata                               0x0800419c   Section      177  usb_desc.o(.constdata)
    .constdata                               0x08004250   Section       44  usb_endp.o(.constdata)
    banbe                                    0x08004250   Data          32  usb_endp.o(.constdata)
    .data                                    0x20000000   Section       20  stm32f10x_rcc.o(.data)
    APBAHBPrescTable                         0x20000000   Data          16  stm32f10x_rcc.o(.data)
    ADCPrescTable                            0x20000010   Data           4  stm32f10x_rcc.o(.data)
    .data                                    0x20000014   Section        8  stm32f10x_it.o(.data)
    .data                                    0x2000001c   Section       26  usb_desc.o(.data)
    .data                                    0x20000038   Section       16  usb_endp.o(.data)
    .data                                    0x20000048   Section       62  usb_istr.o(.data)
    .data                                    0x20000088   Section      148  usb_prop.o(.data)
    .data                                    0x2000011c   Section        7  usb_pwr.o(.data)
    .data                                    0x20000124   Section        4  usb_core.o(.data)
    .data                                    0x20000128   Section       20  usb_init.o(.data)
    .data                                    0x2000013c   Section        4  usb_int.o(.data)
    .data                                    0x20000140   Section        8  rand.o(.data)
    _random_j                                0x20000140   Data           4  rand.o(.data)
    _random_k                                0x20000144   Data           4  rand.o(.data)
    .bss                                     0x20000148   Section    16549  usb_endp.o(.bss)
    .bss                                     0x200041f0   Section       28  usb_init.o(.bss)
    .bss                                     0x2000420c   Section      220  rand.o(.bss)
    _random_number_seed                      0x2000420c   Data         220  rand.o(.bss)
    .bss                                     0x200042e8   Section       96  libspace.o(.bss)
    HEAP                                     0x20004348   Section        0  startup_stm32f10x_md.o(HEAP)
    STACK                                    0x20004348   Section      512  startup_stm32f10x_md.o(STACK)
    Heap_Mem                                 0x20004348   Data           0  startup_stm32f10x_md.o(HEAP)
    Stack_Mem                                0x20004348   Data         512  startup_stm32f10x_md.o(STACK)
    __initial_sp                             0x20004548   Data           0  startup_stm32f10x_md.o(STACK)

    Global Symbols

    Symbol Name                              Value     Ov Type        Size  Object(Section)

    BuildAttributes$$THM_ISAv4$P$D$K$B$S$PE$A:L22UL41UL21$X:L11$S22US41US21$IEEE1$IW$USESV6$~STKCKD$USESV7$~SHL$OSPACE$ROPI$EBA8$UX$STANDARDLIB$REQ8$PRES8$EABIv2 0x00000000   Number         0  anon$$obj.o ABSOLUTE
    __ARM_use_no_argv                        0x00000000   Number         0  main.o ABSOLUTE
    __ARM_exceptions_init                     - Undefined Weak Reference
    __alloca_initialize                       - Undefined Weak Reference
    __cpp_initialize__aeabi_                  - Undefined Weak Reference
    __cxa_finalize                            - Undefined Weak Reference
    __rt_locale                               - Undefined Weak Reference
    __sigvec_lookup                           - Undefined Weak Reference
    _atexit_init                              - Undefined Weak Reference
    _call_atexit_fns                          - Undefined Weak Reference
    _clock_init                               - Undefined Weak Reference
    _fp_trap_init                             - Undefined Weak Reference
    _fp_trap_shutdown                         - Undefined Weak Reference
    _get_lc_collate                           - Undefined Weak Reference
    _get_lc_ctype                             - Undefined Weak Reference
    _get_lc_monetary                          - Undefined Weak Reference
    _get_lc_numeric                           - Undefined Weak Reference
    _get_lc_time                              - Undefined Weak Reference
    _getenv_init                              - Undefined Weak Reference
    _handle_redirection                       - Undefined Weak Reference
    _init_alloc                               - Undefined Weak Reference
    _init_user_alloc                          - Undefined Weak Reference
    _initio                                   - Undefined Weak Reference
    _signal_finish                            - Undefined Weak Reference
    _signal_init                              - Undefined Weak Reference
    _terminate_alloc                          - Undefined Weak Reference
    _terminate_user_alloc                     - Undefined Weak Reference
    _terminateio                              - Undefined Weak Reference
    __Vectors_Size                           0x000000ec   Number         0  startup_stm32f10x_md.o ABSOLUTE
    __Vectors                                0x08000000   Data           4  startup_stm32f10x_md.o(RESET)
    __Vectors_End                            0x080000ec   Data           0  startup_stm32f10x_md.o(RESET)
    __main                                   0x080000ed   Thumb Code     8  __main.o(!!!main)
    __scatterload                            0x080000f5   Thumb Code     0  __scatter.o(!!!scatter)
    __scatterload_rt2                        0x080000f5   Thumb Code    44  __scatter.o(!!!scatter)
    __scatterload_rt2_thumb_only             0x080000f5   Thumb Code     0  __scatter.o(!!!scatter)
    __scatterload_null                       0x08000103   Thumb Code     0  __scatter.o(!!!scatter)
    __decompress                             0x08000129   Thumb Code    90  __dczerorl2.o(!!dczerorl2)
    __decompress1                            0x08000129   Thumb Code     0  __dczerorl2.o(!!dczerorl2)
    __scatterload_zeroinit                   0x08000185   Thumb Code    28  __scatter_zi.o(!!handler_zi)
    __rt_lib_init                            0x080001a1   Thumb Code     0  libinit.o(.ARM.Collect$$libinit$$00000000)
    __rt_lib_init_heap_1                     0x080001a7   Thumb Code     0  libinit2.o(.ARM.Collect$$libinit$$00000006)
    __rt_lib_init_rand_2                     0x080001a7   Thumb Code     0  libinit2.o(.ARM.Collect$$libinit$$00000009)
    __rt_lib_init_user_alloc_1               0x080001a7   Thumb Code     0  libinit2.o(.ARM.Collect$$libinit$$00000008)
    __rt_lib_init_alloca_1                   0x080001ab   Thumb Code     0  libinit2.o(.ARM.Collect$$libinit$$0000002A)
    __rt_lib_init_argv_1                     0x080001ab   Thumb Code     0  libinit2.o(.ARM.Collect$$libinit$$00000028)
    __rt_lib_init_atexit_1                   0x080001ab   Thumb Code     0  libinit2.o(.ARM.Collect$$libinit$$00000017)
    __rt_lib_init_clock_1                    0x080001ab   Thumb Code     0  libinit2.o(.ARM.Collect$$libinit$$0000001D)
    __rt_lib_init_cpp_1                      0x080001ab   Thumb Code     0  libinit2.o(.ARM.Collect$$libinit$$0000002E)
    __rt_lib_init_exceptions_1               0x080001ab   Thumb Code     0  libinit2.o(.ARM.Collect$$libinit$$0000002C)
    __rt_lib_init_fp_trap_1                  0x080001ab   Thumb Code     0  libinit2.o(.ARM.Collect$$libinit$$0000001B)
    __rt_lib_init_getenv_1                   0x080001ab   Thumb Code     0  libinit2.o(.ARM.Collect$$libinit$$0000001F)
    __rt_lib_init_lc_collate_1               0x080001ab   Thumb Code     0  libinit2.o(.ARM.Collect$$libinit$$0000000D)
    __rt_lib_init_lc_ctype_1                 0x080001ab   Thumb Code     0  libinit2.o(.ARM.Collect$$libinit$$0000000F)
    __rt_lib_init_lc_monetary_1              0x080001ab   Thumb Code     0  libinit2.o(.ARM.Collect$$libinit$$00000011)
    __rt_lib_init_lc_numeric_1               0x080001ab   Thumb Code     0  libinit2.o(.ARM.Collect$$libinit$$00000013)
    __rt_lib_init_lc_time_1                  0x080001ab   Thumb Code     0  libinit2.o(.ARM.Collect$$libinit$$00000015)
    __rt_lib_init_rand_1                     0x080001ab   Thumb Code     0  libinit2.o(.ARM.Collect$$libinit$$0000000A)
    __rt_lib_init_return                     0x080001ab   Thumb Code     0  libinit2.o(.ARM.Collect$$libinit$$0000002F)
    __rt_lib_init_signal_1                   0x080001ab   Thumb Code     0  libinit2.o(.ARM.Collect$$libinit$$00000019)
    __rt_lib_init_stdio_1                    0x080001ab   Thumb Code     0  libinit2.o(.ARM.Collect$$libinit$$00000021)
    __rt_lib_shutdown                        0x080001ad   Thumb Code     0  libshutdown.o(.ARM.Collect$$libshutdown$$00000000)
    __rt_lib_shutdown_fp_trap_1              0x080001af   Thumb Code     0  libshutdown2.o(.ARM.Collect$$libshutdown$$00000006)
    __rt_lib_shutdown_heap_1                 0x080001af   Thumb Code     0  libshutdown2.o(.ARM.Collect$$libshutdown$$0000000E)
    __rt_lib_shutdown_return                 0x080001af   Thumb Code     0  libshutdown2.o(.ARM.Collect$$libshutdown$$0000000F)
    __rt_lib_shutdown_signal_1               0x080001af   Thumb Code     0  libshutdown2.o(.ARM.Collect$$libshutdown$$00000009)
    __rt_lib_shutdown_stdio_1                0x080001af   Thumb Code     0  libshutdown2.o(.ARM.Collect$$libshutdown$$00000003)
    __rt_lib_shutdown_user_alloc_1           0x080001af   Thumb Code     0  libshutdown2.o(.ARM.Collect$$libshutdown$$0000000B)
    __rt_entry                               0x080001b1   Thumb Code     0  rtentry.o(.ARM.Collect$$rtentry$$00000000)
    __rt_entry_presh_1                       0x080001b1   Thumb Code     0  rtentry2.o(.ARM.Collect$$rtentry$$00000002)
    __rt_entry_sh                            0x080001b1   Thumb Code     0  rtentry4.o(.ARM.Collect$$rtentry$$00000004)
    __rt_entry_li                            0x080001b7   Thumb Code     0  rtentry2.o(.ARM.Collect$$rtentry$$0000000A)
    __rt_entry_postsh_1                      0x080001b7   Thumb Code     0  rtentry2.o(.ARM.Collect$$rtentry$$00000009)
    __rt_entry_main                          0x080001bb   Thumb Code     0  rtentry2.o(.ARM.Collect$$rtentry$$0000000D)
    __rt_entry_postli_1                      0x080001bb   Thumb Code     0  rtentry2.o(.ARM.Collect$$rtentry$$0000000C)
    __rt_exit                                0x080001c3   Thumb Code     0  rtexit.o(.ARM.Collect$$rtexit$$00000000)
    __rt_exit_ls                             0x080001c3   Thumb Code     0  rtexit2.o(.ARM.Collect$$rtexit$$00000003)
    __rt_exit_prels_1                        0x080001c3   Thumb Code     0  rtexit2.o(.ARM.Collect$$rtexit$$00000002)
    __rt_exit_exit                           0x080001c7   Thumb Code     0  rtexit2.o(.ARM.Collect$$rtexit$$00000004)
    NVIC_PriorityGroupConfig                 0x080001cd   Thumb Code    10  misc.o(.text)
    NVIC_Init                                0x080001d7   Thumb Code   102  misc.o(.text)
    NVIC_SetVectorTable                      0x0800023d   Thumb Code    14  misc.o(.text)
    NVIC_SystemLPConfig                      0x0800024b   Thumb Code    38  misc.o(.text)
    SysTick_CLKSourceConfig                  0x08000271   Thumb Code    40  misc.o(.text)
    ADC_DeInit                               0x080002ad   Thumb Code    90  stm32f10x_adc.o(.text)
    ADC_Init                                 0x08000307   Thumb Code    68  stm32f10x_adc.o(.text)
    ADC_StructInit                           0x0800034b   Thumb Code    18  stm32f10x_adc.o(.text)
    ADC_Cmd                                  0x0800035d   Thumb Code    22  stm32f10x_adc.o(.text)
    ADC_DMACmd                               0x08000373   Thumb Code    22  stm32f10x_adc.o(.text)
    ADC_ITConfig                             0x08000389   Thumb Code    24  stm32f10x_adc.o(.text)
    ADC_ResetCalibration                     0x080003a1   Thumb Code    10  stm32f10x_adc.o(.text)
    ADC_GetResetCalibrationStatus            0x080003ab   Thumb Code    20  stm32f10x_adc.o(.text)
    ADC_StartCalibration                     0x080003bf   Thumb Code    10  stm32f10x_adc.o(.text)
    ADC_GetCalibrationStatus                 0x080003c9   Thumb Code    20  stm32f10x_adc.o(.text)
    ADC_SoftwareStartConvCmd                 0x080003dd   Thumb Code    22  stm32f10x_adc.o(.text)
    ADC_GetSoftwareStartConvStatus           0x080003f3   Thumb Code    20  stm32f10x_adc.o(.text)
    ADC_DiscModeChannelCountConfig           0x08000407   Thumb Code    22  stm32f10x_adc.o(.text)
    ADC_DiscModeCmd                          0x0800041d   Thumb Code    22  stm32f10x_adc.o(.text)
    ADC_RegularChannelConfig                 0x08000433   Thumb Code   180  stm32f10x_adc.o(.text)
    ADC_ExternalTrigConvCmd                  0x080004e7   Thumb Code    22  stm32f10x_adc.o(.text)
    ADC_GetConversionValue                   0x080004fd   Thumb Code     8  stm32f10x_adc.o(.text)
    ADC_GetDualModeConversionValue           0x08000505   Thumb Code     6  stm32f10x_adc.o(.text)
    ADC_AutoInjectedConvCmd                  0x0800050b   Thumb Code    22  stm32f10x_adc.o(.text)
    ADC_InjectedDiscModeCmd                  0x08000521   Thumb Code    22  stm32f10x_adc.o(.text)
    ADC_ExternalTrigInjectedConvConfig       0x08000537   Thumb Code    14  stm32f10x_adc.o(.text)
    ADC_ExternalTrigInjectedConvCmd          0x08000545   Thumb Code    22  stm32f10x_adc.o(.text)
    ADC_SoftwareStartInjectedConvCmd         0x0800055b   Thumb Code    22  stm32f10x_adc.o(.text)
    ADC_GetSoftwareStartInjectedConvCmdStatus 0x08000571   Thumb Code    20  stm32f10x_adc.o(.text)
    ADC_InjectedChannelConfig                0x08000585   Thumb Code   126  stm32f10x_adc.o(.text)
    ADC_InjectedSequencerLengthConfig        0x08000603   Thumb Code    22  stm32f10x_adc.o(.text)
    ADC_SetInjectedOffset                    0x08000619   Thumb Code     4  stm32f10x_adc.o(.text)
    ADC_GetInjectedConversionValue           0x0800061d   Thumb Code    10  stm32f10x_adc.o(.text)
    ADC_AnalogWatchdogCmd                    0x08000627   Thumb Code    14  stm32f10x_adc.o(.text)
    ADC_AnalogWatchdogThresholdsConfig       0x08000635   Thumb Code     6  stm32f10x_adc.o(.text)
    ADC_AnalogWatchdogSingleChannelConfig    0x0800063b   Thumb Code    14  stm32f10x_adc.o(.text)
    ADC_TempSensorVrefintCmd                 0x08000649   Thumb Code    38  stm32f10x_adc.o(.text)
    ADC_GetFlagStatus                        0x0800066f   Thumb Code    18  stm32f10x_adc.o(.text)
    ADC_ClearFlag                            0x08000681   Thumb Code     6  stm32f10x_adc.o(.text)
    ADC_GetITStatus                          0x08000687   Thumb Code    62  stm32f10x_adc.o(.text)
    ADC_ClearITPendingBit                    0x080006c5   Thumb Code    10  stm32f10x_adc.o(.text)
    DMA_DeInit                               0x080006d1   Thumb Code   326  stm32f10x_dma.o(.text)
    DMA_Init                                 0x08000817   Thumb Code    60  stm32f10x_dma.o(.text)
    DMA_StructInit                           0x08000853   Thumb Code    26  stm32f10x_dma.o(.text)
    DMA_Cmd                                  0x0800086d   Thumb Code    22  stm32f10x_dma.o(.text)
    DMA_ITConfig                             0x08000883   Thumb Code    18  stm32f10x_dma.o(.text)
    DMA_GetCurrDataCounter                   0x08000895   Thumb Code     8  stm32f10x_dma.o(.text)
    DMA_GetFlagStatus                        0x0800089d   Thumb Code    38  stm32f10x_dma.o(.text)
    DMA_ClearFlag                            0x080008c3   Thumb Code    20  stm32f10x_dma.o(.text)
    DMA_GetITStatus                          0x080008d7   Thumb Code    38  stm32f10x_dma.o(.text)
    DMA_ClearITPendingBit                    0x080008fd   Thumb Code    20  stm32f10x_dma.o(.text)
    FLASH_SetLatency                         0x08000921   Thumb Code    16  stm32f10x_flash.o(.text)
    FLASH_HalfCycleAccessCmd                 0x08000931   Thumb Code    22  stm32f10x_flash.o(.text)
    FLASH_PrefetchBufferCmd                  0x08000947   Thumb Code    22  stm32f10x_flash.o(.text)
    FLASH_Unlock                             0x0800095d   Thumb Code    12  stm32f10x_flash.o(.text)
    FLASH_Lock                               0x08000969   Thumb Code    14  stm32f10x_flash.o(.text)
    FLASH_GetStatus                          0x08000977   Thumb Code    50  stm32f10x_flash.o(.text)
    FLASH_WaitForLastOperation               0x080009b7   Thumb Code    42  stm32f10x_flash.o(.text)
    FLASH_ErasePage                          0x080009e1   Thumb Code    76  stm32f10x_flash.o(.text)
    FLASH_EraseAllPages                      0x08000a2d   Thumb Code    72  stm32f10x_flash.o(.text)
    FLASH_EraseOptionBytes                   0x08000a75   Thumb Code   142  stm32f10x_flash.o(.text)
    FLASH_ProgramWord                        0x08000b03   Thumb Code   100  stm32f10x_flash.o(.text)
    FLASH_ProgramHalfWord                    0x08000b67   Thumb Code    64  stm32f10x_flash.o(.text)
    FLASH_ProgramOptionByteData              0x08000ba7   Thumb Code    72  stm32f10x_flash.o(.text)
    FLASH_EnableWriteProtection              0x08000bef   Thumb Code   188  stm32f10x_flash.o(.text)
    FLASH_ReadOutProtection                  0x08000cab   Thumb Code   176  stm32f10x_flash.o(.text)
    FLASH_UserOptionByteConfig               0x08000d5b   Thumb Code    94  stm32f10x_flash.o(.text)
    FLASH_GetUserOptionByte                  0x08000db9   Thumb Code     8  stm32f10x_flash.o(.text)
    FLASH_GetWriteProtectionOptionByte       0x08000dc1   Thumb Code     6  stm32f10x_flash.o(.text)
    FLASH_GetReadOutProtectionStatus         0x08000dc7   Thumb Code    20  stm32f10x_flash.o(.text)
    FLASH_GetPrefetchBufferStatus            0x08000ddb   Thumb Code    20  stm32f10x_flash.o(.text)
    FLASH_ITConfig                           0x08000def   Thumb Code    26  stm32f10x_flash.o(.text)
    FLASH_GetFlagStatus                      0x08000e09   Thumb Code    42  stm32f10x_flash.o(.text)
    FLASH_ClearFlag                          0x08000e33   Thumb Code     6  stm32f10x_flash.o(.text)
    GPIO_DeInit                              0x08000e49   Thumb Code   188  stm32f10x_gpio.o(.text)
    GPIO_AFIODeInit                          0x08000f05   Thumb Code    20  stm32f10x_gpio.o(.text)
    GPIO_Init                                0x08000f19   Thumb Code   268  stm32f10x_gpio.o(.text)
    GPIO_StructInit                          0x08001025   Thumb Code    16  stm32f10x_gpio.o(.text)
    GPIO_ReadInputDataBit                    0x08001035   Thumb Code    18  stm32f10x_gpio.o(.text)
    GPIO_ReadInputData                       0x08001047   Thumb Code     8  stm32f10x_gpio.o(.text)
    GPIO_ReadOutputDataBit                   0x0800104f   Thumb Code    18  stm32f10x_gpio.o(.text)
    GPIO_ReadOutputData                      0x08001061   Thumb Code     8  stm32f10x_gpio.o(.text)
    GPIO_SetBits                             0x08001069   Thumb Code     4  stm32f10x_gpio.o(.text)
    GPIO_ResetBits                           0x0800106d   Thumb Code     4  stm32f10x_gpio.o(.text)
    GPIO_WriteBit                            0x08001071   Thumb Code    10  stm32f10x_gpio.o(.text)
    GPIO_Write                               0x0800107b   Thumb Code     4  stm32f10x_gpio.o(.text)
    GPIO_PinLockConfig                       0x0800107f   Thumb Code    18  stm32f10x_gpio.o(.text)
    GPIO_EventOutputConfig                   0x08001091   Thumb Code    24  stm32f10x_gpio.o(.text)
    GPIO_EventOutputCmd                      0x080010a9   Thumb Code     6  stm32f10x_gpio.o(.text)
    GPIO_PinRemapConfig                      0x080010af   Thumb Code   104  stm32f10x_gpio.o(.text)
    GPIO_EXTILineConfig                      0x08001117   Thumb Code    60  stm32f10x_gpio.o(.text)
    RCC_DeInit                               0x08001165   Thumb Code    62  stm32f10x_rcc.o(.text)
    RCC_HSEConfig                            0x080011a3   Thumb Code    70  stm32f10x_rcc.o(.text)
    RCC_GetFlagStatus                        0x080011e9   Thumb Code    56  stm32f10x_rcc.o(.text)
    RCC_WaitForHSEStartUp                    0x08001221   Thumb Code    46  stm32f10x_rcc.o(.text)
    RCC_AdjustHSICalibrationValue            0x0800124f   Thumb Code    18  stm32f10x_rcc.o(.text)
    RCC_HSICmd                               0x08001261   Thumb Code     6  stm32f10x_rcc.o(.text)
    RCC_PLLConfig                            0x08001267   Thumb Code    22  stm32f10x_rcc.o(.text)
    RCC_PLLCmd                               0x0800127d   Thumb Code     6  stm32f10x_rcc.o(.text)
    RCC_SYSCLKConfig                         0x08001283   Thumb Code    16  stm32f10x_rcc.o(.text)
    RCC_GetSYSCLKSource                      0x08001293   Thumb Code    10  stm32f10x_rcc.o(.text)
    RCC_HCLKConfig                           0x0800129d   Thumb Code    16  stm32f10x_rcc.o(.text)
    RCC_PCLK1Config                          0x080012ad   Thumb Code    16  stm32f10x_rcc.o(.text)
    RCC_PCLK2Config                          0x080012bd   Thumb Code    18  stm32f10x_rcc.o(.text)
    RCC_ITConfig                             0x080012cf   Thumb Code    30  stm32f10x_rcc.o(.text)
    RCC_USBCLKConfig                         0x080012ed   Thumb Code     8  stm32f10x_rcc.o(.text)
    RCC_ADCCLKConfig                         0x080012f5   Thumb Code    16  stm32f10x_rcc.o(.text)
    RCC_LSEConfig                            0x08001305   Thumb Code    50  stm32f10x_rcc.o(.text)
    RCC_LSICmd                               0x08001337   Thumb Code     6  stm32f10x_rcc.o(.text)
    RCC_RTCCLKConfig                         0x0800133d   Thumb Code    12  stm32f10x_rcc.o(.text)
    RCC_RTCCLKCmd                            0x08001349   Thumb Code     8  stm32f10x_rcc.o(.text)
    RCC_GetClocksFreq                        0x08001351   Thumb Code   194  stm32f10x_rcc.o(.text)
    RCC_AHBPeriphClockCmd                    0x08001413   Thumb Code    26  stm32f10x_rcc.o(.text)
    RCC_APB2PeriphClockCmd                   0x0800142d   Thumb Code    26  stm32f10x_rcc.o(.text)
    RCC_APB1PeriphClockCmd                   0x08001447   Thumb Code    26  stm32f10x_rcc.o(.text)
    RCC_APB2PeriphResetCmd                   0x08001461   Thumb Code    26  stm32f10x_rcc.o(.text)
    RCC_APB1PeriphResetCmd                   0x0800147b   Thumb Code    26  stm32f10x_rcc.o(.text)
    RCC_BackupResetCmd                       0x08001495   Thumb Code     8  stm32f10x_rcc.o(.text)
    RCC_ClockSecuritySystemCmd               0x0800149d   Thumb Code     6  stm32f10x_rcc.o(.text)
    RCC_MCOConfig                            0x080014a3   Thumb Code     6  stm32f10x_rcc.o(.text)
    RCC_ClearFlag                            0x080014a9   Thumb Code    14  stm32f10x_rcc.o(.text)
    RCC_GetITStatus                          0x080014b7   Thumb Code    20  stm32f10x_rcc.o(.text)
    RCC_ClearITPendingBit                    0x080014cb   Thumb Code     6  stm32f10x_rcc.o(.text)
    GPIO_configure                           0x080014f1   Thumb Code    84  main.o(.text)
    Set_System                               0x08001545   Thumb Code   106  main.o(.text)
    main                                     0x080015af   Thumb Code   102  main.o(.text)
    Delay                                    0x08001615   Thumb Code    10  main.o(.text)
    Callback                                 0x0800161f   Thumb Code    78  main.o(.text)
    NMI_Handler                              0x08001679   Thumb Code     2  stm32f10x_it.o(.text)
    HardFault_Handler                        0x0800167b   Thumb Code     4  stm32f10x_it.o(.text)
    MemManage_Handler                        0x0800167f   Thumb Code     4  stm32f10x_it.o(.text)
    BusFault_Handler                         0x08001683   Thumb Code     4  stm32f10x_it.o(.text)
    UsageFault_Handler                       0x08001687   Thumb Code     4  stm32f10x_it.o(.text)
    SVC_Handler                              0x0800168b   Thumb Code     2  stm32f10x_it.o(.text)
    DebugMon_Handler                         0x0800168d   Thumb Code     2  stm32f10x_it.o(.text)
    PendSV_Handler                           0x0800168f   Thumb Code     2  stm32f10x_it.o(.text)
    SysTick_Handler                          0x08001691   Thumb Code     2  stm32f10x_it.o(.text)
    DMA1_Channel1_IRQHandler                 0x08001693   Thumb Code   492  stm32f10x_it.o(.text)
    USB_HP_CAN1_TX_IRQHandler                0x0800187f   Thumb Code    16  stm32f10x_it.o(.text)
    USB_LP_CAN1_RX0_IRQHandler               0x0800188f   Thumb Code     8  stm32f10x_it.o(.text)
    USART1_IRQHandler                        0x08001897   Thumb Code     2  stm32f10x_it.o(.text)
    USART2_IRQHandler                        0x08001899   Thumb Code     2  stm32f10x_it.o(.text)
    USB_GPIO_Config                          0x080018c1   Thumb Code    40  qdmx_usb.o(.text)
    Set_USBClock                             0x080018e9   Thumb Code    18  qdmx_usb.o(.text)
    USB_Interrupts_Config                    0x080018fb   Thumb Code    40  qdmx_usb.o(.text)
    Enter_LowPowerMode                       0x08001923   Thumb Code     8  qdmx_usb.o(.text)
    Leave_LowPowerMode                       0x0800192b   Thumb Code    22  qdmx_usb.o(.text)
    USB_Cable_Config                         0x08001941   Thumb Code    30  qdmx_usb.o(.text)
    Get_SerialNum                            0x0800195f   Thumb Code    66  qdmx_usb.o(.text)
    EP1_IN_Callback                          0x080019b9   Thumb Code   114  usb_endp.o(.text)
    EP3_OUT_Callback                         0x08001a2b   Thumb Code  1150  usb_endp.o(.text)
    USB_Istr                                 0x08001ec1   Thumb Code   120  usb_istr.o(.text)
    Virtual_Com_Port_init                    0x08001f4d   Thumb Code    30  usb_prop.o(.text)
    Virtual_Com_Port_Reset                   0x08001f6b   Thumb Code   254  usb_prop.o(.text)
    Virtual_Com_Port_SetConfiguration        0x08002069   Thumb Code    14  usb_prop.o(.text)
    Virtual_Com_Port_SetDeviceAddress        0x08002077   Thumb Code     8  usb_prop.o(.text)
    Virtual_Com_Port_Status_In               0x0800207f   Thumb Code    16  usb_prop.o(.text)
    Virtual_Com_Port_Status_Out              0x0800208f   Thumb Code     2  usb_prop.o(.text)
    Virtual_Com_Port_SetLineCoding           0x08002091   Thumb Code    20  usb_prop.o(.text)
    Virtual_Com_Port_GetLineCoding           0x080020a5   Thumb Code    20  usb_prop.o(.text)
    Virtual_Com_Port_Data_Setup              0x080020b9   Thumb Code    86  usb_prop.o(.text)
    Virtual_Com_Port_NoData_Setup            0x0800210f   Thumb Code    36  usb_prop.o(.text)
    Virtual_Com_Port_GetDeviceDescriptor     0x08002133   Thumb Code    14  usb_prop.o(.text)
    Virtual_Com_Port_GetConfigDescriptor     0x08002141   Thumb Code    14  usb_prop.o(.text)
    Virtual_Com_Port_GetStringDescriptor     0x0800214f   Thumb Code    32  usb_prop.o(.text)
    Virtual_Com_Port_Get_Interface_Setting   0x0800216f   Thumb Code    22  usb_prop.o(.text)
    PowerOn                                  0x080021ad   Thumb Code    60  usb_pwr.o(.text)
    PowerOff                                 0x080021e9   Thumb Code    30  usb_pwr.o(.text)
    Suspend                                  0x08002207   Thumb Code    40  usb_pwr.o(.text)
    Resume_Init                              0x0800222f   Thumb Code    32  usb_pwr.o(.text)
    Resume                                   0x0800224f   Thumb Code   172  usb_pwr.o(.text)
    m_adc_clk_config                         0x0800230d   Thumb Code    28  qdmx_adc.o(.text)
    m_adc_gpio_config                        0x08002329   Thumb Code    32  qdmx_adc.o(.text)
    m_adc_init                               0x08002349   Thumb Code   228  qdmx_adc.o(.text)
    m_adc_Interrupts_Config                  0x0800242d   Thumb Code    28  qdmx_adc.o(.text)
    Control_a                                0x08002449   Thumb Code   518  qdmx_adc.o(.text)
    Control_b                                0x0800264f   Thumb Code   514  qdmx_adc.o(.text)
    Reset_Handler                            0x08002859   Thumb Code     4  startup_stm32f10x_md.o(.text)
    ADC1_2_IRQHandler                        0x0800286f   Thumb Code     0  startup_stm32f10x_md.o(.text)
    CAN1_RX1_IRQHandler                      0x0800286f   Thumb Code     0  startup_stm32f10x_md.o(.text)
    CAN1_SCE_IRQHandler                      0x0800286f   Thumb Code     0  startup_stm32f10x_md.o(.text)
    DMA1_Channel2_IRQHandler                 0x0800286f   Thumb Code     0  startup_stm32f10x_md.o(.text)
    DMA1_Channel3_IRQHandler                 0x0800286f   Thumb Code     0  startup_stm32f10x_md.o(.text)
    DMA1_Channel4_IRQHandler                 0x0800286f   Thumb Code     0  startup_stm32f10x_md.o(.text)
    DMA1_Channel5_IRQHandler                 0x0800286f   Thumb Code     0  startup_stm32f10x_md.o(.text)
    DMA1_Channel6_IRQHandler                 0x0800286f   Thumb Code     0  startup_stm32f10x_md.o(.text)
    DMA1_Channel7_IRQHandler                 0x0800286f   Thumb Code     0  startup_stm32f10x_md.o(.text)
    EXTI0_IRQHandler                         0x0800286f   Thumb Code     0  startup_stm32f10x_md.o(.text)
    EXTI15_10_IRQHandler                     0x0800286f   Thumb Code     0  startup_stm32f10x_md.o(.text)
    EXTI1_IRQHandler                         0x0800286f   Thumb Code     0  startup_stm32f10x_md.o(.text)
    EXTI2_IRQHandler                         0x0800286f   Thumb Code     0  startup_stm32f10x_md.o(.text)
    EXTI3_IRQHandler                         0x0800286f   Thumb Code     0  startup_stm32f10x_md.o(.text)
    EXTI4_IRQHandler                         0x0800286f   Thumb Code     0  startup_stm32f10x_md.o(.text)
    EXTI9_5_IRQHandler                       0x0800286f   Thumb Code     0  startup_stm32f10x_md.o(.text)
    FLASH_IRQHandler                         0x0800286f   Thumb Code     0  startup_stm32f10x_md.o(.text)
    I2C1_ER_IRQHandler                       0x0800286f   Thumb Code     0  startup_stm32f10x_md.o(.text)
    I2C1_EV_IRQHandler                       0x0800286f   Thumb Code     0  startup_stm32f10x_md.o(.text)
    I2C2_ER_IRQHandler                       0x0800286f   Thumb Code     0  startup_stm32f10x_md.o(.text)
    I2C2_EV_IRQHandler                       0x0800286f   Thumb Code     0  startup_stm32f10x_md.o(.text)
    PVD_IRQHandler                           0x0800286f   Thumb Code     0  startup_stm32f10x_md.o(.text)
    RCC_IRQHandler                           0x0800286f   Thumb Code     0  startup_stm32f10x_md.o(.text)
    RTCAlarm_IRQHandler                      0x0800286f   Thumb Code     0  startup_stm32f10x_md.o(.text)
    RTC_IRQHandler                           0x0800286f   Thumb Code     0  startup_stm32f10x_md.o(.text)
    SPI1_IRQHandler                          0x0800286f   Thumb Code     0  startup_stm32f10x_md.o(.text)
    SPI2_IRQHandler                          0x0800286f   Thumb Code     0  startup_stm32f10x_md.o(.text)
    TAMPER_IRQHandler                        0x0800286f   Thumb Code     0  startup_stm32f10x_md.o(.text)
    TIM1_BRK_IRQHandler                      0x0800286f   Thumb Code     0  startup_stm32f10x_md.o(.text)
    TIM1_CC_IRQHandler                       0x0800286f   Thumb Code     0  startup_stm32f10x_md.o(.text)
    TIM1_TRG_COM_IRQHandler                  0x0800286f   Thumb Code     0  startup_stm32f10x_md.o(.text)
    TIM1_UP_IRQHandler                       0x0800286f   Thumb Code     0  startup_stm32f10x_md.o(.text)
    TIM2_IRQHandler                          0x0800286f   Thumb Code     0  startup_stm32f10x_md.o(.text)
    TIM3_IRQHandler                          0x0800286f   Thumb Code     0  startup_stm32f10x_md.o(.text)
    TIM4_IRQHandler                          0x0800286f   Thumb Code     0  startup_stm32f10x_md.o(.text)
    USART3_IRQHandler                        0x0800286f   Thumb Code     0  startup_stm32f10x_md.o(.text)
    USBWakeUp_IRQHandler                     0x0800286f   Thumb Code     0  startup_stm32f10x_md.o(.text)
    WWDG_IRQHandler                          0x0800286f   Thumb Code     0  startup_stm32f10x_md.o(.text)
    __user_initial_stackheap                 0x08002871   Thumb Code     0  startup_stm32f10x_md.o(.text)
    Standard_GetConfiguration                0x0800288d   Thumb Code    34  usb_core.o(.text)
    Standard_SetConfiguration                0x080028af   Thumb Code    60  usb_core.o(.text)
    Standard_GetInterface                    0x080028eb   Thumb Code    34  usb_core.o(.text)
    Standard_SetInterface                    0x0800290d   Thumb Code    96  usb_core.o(.text)
    Standard_GetStatus                       0x0800296d   Thumb Code   238  usb_core.o(.text)
    Standard_ClearFeature                    0x08002a5b   Thumb Code   338  usb_core.o(.text)
    Standard_SetEndPointFeature              0x08002bad   Thumb Code   228  usb_core.o(.text)
    Standard_SetDeviceFeature                0x08002c91   Thumb Code    30  usb_core.o(.text)
    Standard_GetDescriptorData               0x08002caf   Thumb Code    32  usb_core.o(.text)
    Post0_Process                            0x080031e5   Thumb Code    56  usb_core.o(.text)
    Setup0_Process                           0x0800321d   Thumb Code   170  usb_core.o(.text)
    SetDeviceAddress                         0x080032c7   Thumb Code    70  usb_core.o(.text)
    In0_Process                              0x0800330d   Thumb Code    98  usb_core.o(.text)
    Out0_Process                             0x0800336f   Thumb Code    70  usb_core.o(.text)
    NOP_Process                              0x080033b5   Thumb Code     2  usb_core.o(.text)
    USB_Init                                 0x080033e5   Thumb Code    36  usb_init.o(.text)
    CTR_LP                                   0x08003421   Thumb Code   610  usb_int.o(.text)
    CTR_HP                                   0x08003683   Thumb Code   178  usb_int.o(.text)
    UserToPMABufferCopy                      0x08003755   Thumb Code    50  usb_mem.o(.text)
    PMAToUserBufferCopy                      0x08003787   Thumb Code    32  usb_mem.o(.text)
    SetCNTR                                  0x080037ad   Thumb Code     6  usb_regs.o(.text)
    GetCNTR                                  0x080037b3   Thumb Code     8  usb_regs.o(.text)
    SetISTR                                  0x080037bb   Thumb Code     8  usb_regs.o(.text)
    GetISTR                                  0x080037c3   Thumb Code    10  usb_regs.o(.text)
    GetFNR                                   0x080037cd   Thumb Code    10  usb_regs.o(.text)
    SetDADDR                                 0x080037d7   Thumb Code     8  usb_regs.o(.text)
    GetDADDR                                 0x080037df   Thumb Code    10  usb_regs.o(.text)
    SetBTABLE                                0x080037e9   Thumb Code    14  usb_regs.o(.text)
    GetBTABLE                                0x080037f7   Thumb Code    10  usb_regs.o(.text)
    SetENDPOINT                              0x08003801   Thumb Code    12  usb_regs.o(.text)
    GetENDPOINT                              0x0800380d   Thumb Code    16  usb_regs.o(.text)
    SetEPType                                0x0800381d   Thumb Code    32  usb_regs.o(.text)
    GetEPType                                0x0800383d   Thumb Code    18  usb_regs.o(.text)
    SetEPTxStatus                            0x0800384f   Thumb Code    62  usb_regs.o(.text)
    SetEPRxStatus                            0x0800388d   Thumb Code    62  usb_regs.o(.text)
    SetDouBleBuffEPStall                     0x080038cb   Thumb Code    54  usb_regs.o(.text)
    GetEPTxStatus                            0x08003901   Thumb Code    18  usb_regs.o(.text)
    GetEPRxStatus                            0x08003913   Thumb Code    18  usb_regs.o(.text)
    SetEPTxValid                             0x08003925   Thumb Code    48  usb_regs.o(.text)
    SetEPRxValid                             0x08003955   Thumb Code    48  usb_regs.o(.text)
    SetEP_KIND                               0x08003985   Thumb Code    40  usb_regs.o(.text)
    ClearEP_KIND                             0x080039ad   Thumb Code    36  usb_regs.o(.text)
    Clear_Status_Out                         0x080039d1   Thumb Code    36  usb_regs.o(.text)
    Set_Status_Out                           0x080039f5   Thumb Code    40  usb_regs.o(.text)
    SetEPDoubleBuff                          0x08003a1d   Thumb Code    40  usb_regs.o(.text)
    ClearEPDoubleBuff                        0x08003a45   Thumb Code    36  usb_regs.o(.text)
    GetTxStallStatus                         0x08003a69   Thumb Code    30  usb_regs.o(.text)
    GetRxStallStatus                         0x08003a87   Thumb Code    32  usb_regs.o(.text)
    ClearEP_CTR_RX                           0x08003aa7   Thumb Code    32  usb_regs.o(.text)
    ClearEP_CTR_TX                           0x08003ac7   Thumb Code    30  usb_regs.o(.text)
    ToggleDTOG_RX                            0x08003ae5   Thumb Code    36  usb_regs.o(.text)
    ToggleDTOG_TX                            0x08003b09   Thumb Code    36  usb_regs.o(.text)
    ClearDTOG_RX                             0x08003b2d   Thumb Code    52  usb_regs.o(.text)
    ClearDTOG_TX                             0x08003b61   Thumb Code    60  usb_regs.o(.text)
    SetEPAddress                             0x08003b9d   Thumb Code    38  usb_regs.o(.text)
    GetEPAddress                             0x08003bc3   Thumb Code    18  usb_regs.o(.text)
    SetEPTxAddr                              0x08003bd5   Thumb Code    24  usb_regs.o(.text)
    SetEPRxAddr                              0x08003bed   Thumb Code    26  usb_regs.o(.text)
    GetEPTxAddr                              0x08003c07   Thumb Code    22  usb_regs.o(.text)
    GetEPRxAddr                              0x08003c1d   Thumb Code    24  usb_regs.o(.text)
    SetEPTxCount                             0x08003c35   Thumb Code    20  usb_regs.o(.text)
    SetEPCountRxReg                          0x08003c49   Thumb Code    46  usb_regs.o(.text)
    SetEPRxCount                             0x08003c77   Thumb Code    66  usb_regs.o(.text)
    GetEPTxCount                             0x08003cb9   Thumb Code    26  usb_regs.o(.text)
    GetEPRxCount                             0x08003cd3   Thumb Code    26  usb_regs.o(.text)
    SetEPDblBuffAddr                         0x08003ced   Thumb Code    46  usb_regs.o(.text)
    SetEPDblBuf0Addr                         0x08003d1b   Thumb Code    24  usb_regs.o(.text)
    SetEPDblBuf1Addr                         0x08003d33   Thumb Code    26  usb_regs.o(.text)
    GetEPDblBuf0Addr                         0x08003d4d   Thumb Code    22  usb_regs.o(.text)
    GetEPDblBuf1Addr                         0x08003d63   Thumb Code    24  usb_regs.o(.text)
    SetEPDblBuffCount                        0x08003d7b   Thumb Code   184  usb_regs.o(.text)
    SetEPDblBuf0Count                        0x08003e33   Thumb Code    94  usb_regs.o(.text)
    SetEPDblBuf1Count                        0x08003e91   Thumb Code    94  usb_regs.o(.text)
    GetEPDblBuf0Count                        0x08003eef   Thumb Code    26  usb_regs.o(.text)
    GetEPDblBuf1Count                        0x08003f09   Thumb Code    26  usb_regs.o(.text)
    GetEPDblBufDir                           0x08003f23   Thumb Code    62  usb_regs.o(.text)
    FreeUserBuffer                           0x08003f61   Thumb Code    92  usb_regs.o(.text)
    ToWord                                   0x08003fbd   Thumb Code     8  usb_regs.o(.text)
    ByteSwap                                 0x08003fc5   Thumb Code    12  usb_regs.o(.text)
    USB_SIL_Init                             0x08003fd5   Thumb Code    28  usb_sil.o(.text)
    USB_SIL_Write                            0x08003ff1   Thumb Code    46  usb_sil.o(.text)
    USB_SIL_Read                             0x0800401f   Thumb Code    46  usb_sil.o(.text)
    srand                                    0x08004059   Thumb Code    40  rand.o(.text)
    _rand_init                               0x08004081   Thumb Code     4  rand.o(.text)
    rand                                     0x08004085   Thumb Code    58  rand.o(.text)
    __aeabi_memclr4                          0x080040d1   Thumb Code     0  rt_memclr_w.o(.text)
    __aeabi_memclr8                          0x080040d1   Thumb Code     0  rt_memclr_w.o(.text)
    __rt_memclr_w                            0x080040d1   Thumb Code    78  rt_memclr_w.o(.text)
    _memset_w                                0x080040d5   Thumb Code     0  rt_memclr_w.o(.text)
    __use_two_region_memory                  0x0800411f   Thumb Code     2  heapauxi.o(.text)
    __rt_heap_escrow$2region                 0x08004121   Thumb Code     2  heapauxi.o(.text)
    __rt_heap_expand$2region                 0x08004123   Thumb Code     2  heapauxi.o(.text)
    __user_setup_stackheap                   0x08004125   Thumb Code    74  sys_stackheap_outer.o(.text)
    exit                                     0x0800416f   Thumb Code    12  exit.o(.text)
    __user_libspace                          0x0800417d   Thumb Code     8  libspace.o(.text)
    __user_perproc_libspace                  0x0800417d   Thumb Code     0  libspace.o(.text)
    __user_perthread_libspace                0x0800417d   Thumb Code     0  libspace.o(.text)
    __I$use$semihosting                      0x08004185   Thumb Code     0  use_no_semi.o(.text)
    __use_no_semihosting_swi                 0x08004185   Thumb Code     2  use_no_semi.o(.text)
    _sys_exit                                0x08004189   Thumb Code    16  sys_exit.o(.text)
    Virtual_Com_Port_DeviceDescriptor        0x0800419c   Data          18  usb_desc.o(.constdata)
    Virtual_Com_Port_ConfigDescriptor        0x080041ae   Data          67  usb_desc.o(.constdata)
    Virtual_Com_Port_StringLangID            0x080041f1   Data           4  usb_desc.o(.constdata)
    Virtual_Com_Port_StringVendor            0x080041f5   Data          38  usb_desc.o(.constdata)
    Virtual_Com_Port_StringProduct           0x0800421b   Data          50  usb_desc.o(.constdata)
    Region$$Table$$Base                      0x0800427c   Number         0  anon$$obj.o(Region$$Table)
    Region$$Table$$Limit                     0x0800429c   Number         0  anon$$obj.o(Region$$Table)
    Controla_a                               0x20000014   Data           1  stm32f10x_it.o(.data)
    Controla_b                               0x20000015   Data           1  stm32f10x_it.o(.data)
    count                                    0x20000018   Data           4  stm32f10x_it.o(.data)
    Virtual_Com_Port_StringSerial            0x2000001c   Data          26  usb_desc.o(.data)
    count_out                                0x20000038   Data           4  usb_endp.o(.data)
    shakesuccess                             0x2000003c   Data           1  usb_endp.o(.data)
    status                                   0x2000003d   Data           1  usb_endp.o(.data)
    csbb                                     0x2000003e   Data           1  usb_endp.o(.data)
    sign                                     0x2000003f   Data           1  usb_endp.o(.data)
    count_in                                 0x20000040   Data           4  usb_endp.o(.data)
    cyl                                      0x20000044   Data           4  usb_endp.o(.data)
    bIntPackSOF                              0x20000048   Data           1  usb_istr.o(.data)
    pEpInt_IN                                0x2000004c   Data          28  usb_istr.o(.data)
    pEpInt_OUT                               0x20000068   Data          28  usb_istr.o(.data)
    wIstr                                    0x20000084   Data           2  usb_istr.o(.data)
    Request                                  0x20000088   Data           1  usb_prop.o(.data)
    linecoding                               0x2000008c   Data           8  usb_prop.o(.data)
    Device_Table                             0x20000094   Data           2  usb_prop.o(.data)
    Device_Property                          0x20000098   Data          48  usb_prop.o(.data)
    User_Standard_Requests                   0x200000c8   Data          36  usb_prop.o(.data)
    Device_Descriptor                        0x200000ec   Data           8  usb_prop.o(.data)
    Config_Descriptor                        0x200000f4   Data           8  usb_prop.o(.data)
    String_Descriptor                        0x200000fc   Data          32  usb_prop.o(.data)
    bDeviceState                             0x2000011c   Data           4  usb_pwr.o(.data)
    fSuspendEnabled                          0x20000120   Data           1  usb_pwr.o(.data)
    ResumeS                                  0x20000121   Data           2  usb_pwr.o(.data)
    Data_Mul_MaxPacketSize                   0x20000124   Data           1  usb_core.o(.data)
    StatusInfo                               0x20000126   Data           2  usb_core.o(.data)
    EPindex                                  0x20000128   Data           1  usb_init.o(.data)
    pInformation                             0x2000012c   Data           4  usb_init.o(.data)
    pProperty                                0x20000130   Data           4  usb_init.o(.data)
    SaveState                                0x20000134   Data           2  usb_init.o(.data)
    wInterrupt_Mask                          0x20000136   Data           2  usb_init.o(.data)
    pUser_Standard_Requests                  0x20000138   Data           4  usb_init.o(.data)
    SaveRState                               0x2000013c   Data           2  usb_int.o(.data)
    SaveTState                               0x2000013e   Data           2  usb_int.o(.data)
    back                                     0x20000148   Data          32  usb_endp.o(.bss)
    b                                        0x20000168   Data          37  usb_endp.o(.bss)
    d                                        0x2000018d   Data          32  usb_endp.o(.bss)
    buffer_out                               0x200001ad   Data          64  usb_endp.o(.bss)
    ADCConvertedValue                        0x200001ed   Data       16384  usb_endp.o(.bss)
    Device_Info                              0x200041f0   Data          28  usb_init.o(.bss)
    __libspace_start                         0x200042e8   Data          96  libspace.o(.bss)
    __temporary_stack_top$libspace           0x20004348   Data           0  libspace.o(.bss)



==============================================================================

Memory Map of the image

  Image Entry point : 0x080000ed

  Load Region LR_IROM1 (Base: 0x08000000, Size: 0x000043e4, Max: 0x00010000, ABSOLUTE, COMPRESSED[0x0000432c])

    Execution Region ER_IROM1 (Base: 0x08000000, Size: 0x0000429c, Max: 0x00010000, ABSOLUTE)

    Base Addr    Size         Type   Attr      Idx    E Section Name        Object

    0x08000000   0x000000ec   Data   RO          468    RESET               startup_stm32f10x_md.o
    0x080000ec   0x00000008   Code   RO          581  * !!!main             __main.o(c_w.l)
    0x080000f4   0x00000034   Code   RO          740    !!!scatter          __scatter.o(c_w.l)
    0x08000128   0x0000005a   Code   RO          738    !!dczerorl2         __dczerorl2.o(c_w.l)
    0x08000182   0x00000002   PAD
    0x08000184   0x0000001c   Code   RO          742    !!handler_zi        __scatter_zi.o(c_w.l)
    0x080001a0   0x00000006   Code   RO          660    .ARM.Collect$$libinit$$00000000  libinit.o(c_w.l)
    0x080001a6   0x00000000   Code   RO          587    .ARM.Collect$$libinit$$00000006  libinit2.o(c_w.l)
    0x080001a6   0x00000000   Code   RO          589    .ARM.Collect$$libinit$$00000008  libinit2.o(c_w.l)
    0x080001a6   0x00000004   Code   RO          590    .ARM.Collect$$libinit$$00000009  libinit2.o(c_w.l)
    0x080001aa   0x00000000   Code   RO          591    .ARM.Collect$$libinit$$0000000A  libinit2.o(c_w.l)
    0x080001aa   0x00000000   Code   RO          594    .ARM.Collect$$libinit$$0000000D  libinit2.o(c_w.l)
    0x080001aa   0x00000000   Code   RO          596    .ARM.Collect$$libinit$$0000000F  libinit2.o(c_w.l)
    0x080001aa   0x00000000   Code   RO          598    .ARM.Collect$$libinit$$00000011  libinit2.o(c_w.l)
    0x080001aa   0x00000000   Code   RO          600    .ARM.Collect$$libinit$$00000013  libinit2.o(c_w.l)
    0x080001aa   0x00000000   Code   RO          602    .ARM.Collect$$libinit$$00000015  libinit2.o(c_w.l)
    0x080001aa   0x00000000   Code   RO          604    .ARM.Collect$$libinit$$00000017  libinit2.o(c_w.l)
    0x080001aa   0x00000000   Code   RO          606    .ARM.Collect$$libinit$$00000019  libinit2.o(c_w.l)
    0x080001aa   0x00000000   Code   RO          608    .ARM.Collect$$libinit$$0000001B  libinit2.o(c_w.l)
    0x080001aa   0x00000000   Code   RO          610    .ARM.Collect$$libinit$$0000001D  libinit2.o(c_w.l)
    0x080001aa   0x00000000   Code   RO          612    .ARM.Collect$$libinit$$0000001F  libinit2.o(c_w.l)
    0x080001aa   0x00000000   Code   RO          614    .ARM.Collect$$libinit$$00000021  libinit2.o(c_w.l)
    0x080001aa   0x00000000   Code   RO          618    .ARM.Collect$$libinit$$00000028  libinit2.o(c_w.l)
    0x080001aa   0x00000000   Code   RO          620    .ARM.Collect$$libinit$$0000002A  libinit2.o(c_w.l)
    0x080001aa   0x00000000   Code   RO          622    .ARM.Collect$$libinit$$0000002C  libinit2.o(c_w.l)
    0x080001aa   0x00000000   Code   RO          624    .ARM.Collect$$libinit$$0000002E  libinit2.o(c_w.l)
    0x080001aa   0x00000002   Code   RO          625    .ARM.Collect$$libinit$$0000002F  libinit2.o(c_w.l)
    0x080001ac   0x00000002   Code   RO          700    .ARM.Collect$$libshutdown$$00000000  libshutdown.o(c_w.l)
    0x080001ae   0x00000000   Code   RO          707    .ARM.Collect$$libshutdown$$00000003  libshutdown2.o(c_w.l)
    0x080001ae   0x00000000   Code   RO          710    .ARM.Collect$$libshutdown$$00000006  libshutdown2.o(c_w.l)
    0x080001ae   0x00000000   Code   RO          713    .ARM.Collect$$libshutdown$$00000009  libshutdown2.o(c_w.l)
    0x080001ae   0x00000000   Code   RO          715    .ARM.Collect$$libshutdown$$0000000B  libshutdown2.o(c_w.l)
    0x080001ae   0x00000000   Code   RO          718    .ARM.Collect$$libshutdown$$0000000E  libshutdown2.o(c_w.l)
    0x080001ae   0x00000002   Code   RO          719    .ARM.Collect$$libshutdown$$0000000F  libshutdown2.o(c_w.l)
    0x080001b0   0x00000000   Code   RO          583    .ARM.Collect$$rtentry$$00000000  rtentry.o(c_w.l)
    0x080001b0   0x00000000   Code   RO          627    .ARM.Collect$$rtentry$$00000002  rtentry2.o(c_w.l)
    0x080001b0   0x00000006   Code   RO          642    .ARM.Collect$$rtentry$$00000004  rtentry4.o(c_w.l)
    0x080001b6   0x00000000   Code   RO          629    .ARM.Collect$$rtentry$$00000009  rtentry2.o(c_w.l)
    0x080001b6   0x00000004   Code   RO          630    .ARM.Collect$$rtentry$$0000000A  rtentry2.o(c_w.l)
    0x080001ba   0x00000000   Code   RO          632    .ARM.Collect$$rtentry$$0000000C  rtentry2.o(c_w.l)
    0x080001ba   0x00000008   Code   RO          633    .ARM.Collect$$rtentry$$0000000D  rtentry2.o(c_w.l)
    0x080001c2   0x00000000   Code   RO          666    .ARM.Collect$$rtexit$$00000000  rtexit.o(c_w.l)
    0x080001c2   0x00000000   Code   RO          679    .ARM.Collect$$rtexit$$00000002  rtexit2.o(c_w.l)
    0x080001c2   0x00000004   Code   RO          680    .ARM.Collect$$rtexit$$00000003  rtexit2.o(c_w.l)
    0x080001c6   0x00000004   Code   RO          681    .ARM.Collect$$rtexit$$00000004  rtexit2.o(c_w.l)
    0x080001ca   0x00000002   PAD
    0x080001cc   0x000000e0   Code   RO            1    .text               misc.o
    0x080002ac   0x00000422   Code   RO           49    .text               stm32f10x_adc.o
    0x080006ce   0x00000002   PAD
    0x080006d0   0x00000250   Code   RO          124    .text               stm32f10x_dma.o
    0x08000920   0x00000528   Code   RO          151    .text               stm32f10x_flash.o
    0x08000e48   0x0000031c   Code   RO          178    .text               stm32f10x_gpio.o
    0x08001164   0x0000038c   Code   RO          220    .text               stm32f10x_rcc.o
    0x080014f0   0x00000188   Code   RO          234    .text               main.o
    0x08001678   0x00000248   Code   RO          294    .text               stm32f10x_it.o
    0x080018c0   0x000000f8   Code   RO          316    .text               qdmx_usb.o
    0x080019b8   0x00000508   Code   RO          341    .text               usb_endp.o
    0x08001ec0   0x0000008c   Code   RO          362    .text               usb_istr.o
    0x08001f4c   0x00000260   Code   RO          383    .text               usb_prop.o
    0x080021ac   0x00000160   Code   RO          406    .text               usb_pwr.o
    0x0800230c   0x0000054c   Code   RO          424    .text               qdmx_adc.o
    0x08002858   0x00000034   Code   RO          469    .text               startup_stm32f10x_md.o
    0x0800288c   0x00000b58   Code   RO          473    .text               usb_core.o
    0x080033e4   0x0000003c   Code   RO          488    .text               usb_init.o
    0x08003420   0x00000334   Code   RO          511    .text               usb_int.o
    0x08003754   0x00000058   Code   RO          535    .text               usb_mem.o
    0x080037ac   0x00000828   Code   RO          547    .text               usb_regs.o
    0x08003fd4   0x00000084   Code   RO          559    .text               usb_sil.o
    0x08004058   0x00000078   Code   RO          573    .text               rand.o(c_w.l)
    0x080040d0   0x0000004e   Code   RO          577    .text               rt_memclr_w.o(c_w.l)
    0x0800411e   0x00000006   Code   RO          579    .text               heapauxi.o(c_w.l)
    0x08004124   0x0000004a   Code   RO          646    .text               sys_stackheap_outer.o(c_w.l)
    0x0800416e   0x0000000c   Code   RO          648    .text               exit.o(c_w.l)
    0x0800417a   0x00000002   PAD
    0x0800417c   0x00000008   Code   RO          663    .text               libspace.o(c_w.l)
    0x08004184   0x00000002   Code   RO          676    .text               use_no_semi.o(c_w.l)
    0x08004186   0x00000002   PAD
    0x08004188   0x00000014   Code   RO          692    .text               sys_exit.o(c_w.l)
    0x0800419c   0x000000b1   Data   RO          328    .constdata          usb_desc.o
    0x0800424d   0x00000003   PAD
    0x08004250   0x0000002c   Data   RO          343    .constdata          usb_endp.o
    0x0800427c   0x00000020   Data   RO          736    Region$$Table       anon$$obj.o


    Execution Region RW_IRAM1 (Base: 0x20000000, Size: 0x00004548, Max: 0x00005000, ABSOLUTE, COMPRESSED[0x00000090])

    Base Addr    Size         Type   Attr      Idx    E Section Name        Object

    0x20000000   0x00000014   Data   RW          221    .data               stm32f10x_rcc.o
    0x20000014   0x00000008   Data   RW          295    .data               stm32f10x_it.o
    0x2000001c   0x0000001a   Data   RW          329    .data               usb_desc.o
    0x20000036   0x00000002   PAD
    0x20000038   0x00000010   Data   RW          344    .data               usb_endp.o
    0x20000048   0x0000003e   Data   RW          363    .data               usb_istr.o
    0x20000086   0x00000002   PAD
    0x20000088   0x00000094   Data   RW          384    .data               usb_prop.o
    0x2000011c   0x00000007   Data   RW          407    .data               usb_pwr.o
    0x20000123   0x00000001   PAD
    0x20000124   0x00000004   Data   RW          474    .data               usb_core.o
    0x20000128   0x00000014   Data   RW          490    .data               usb_init.o
    0x2000013c   0x00000004   Data   RW          512    .data               usb_int.o
    0x20000140   0x00000008   Data   RW          575    .data               rand.o(c_w.l)
    0x20000148   0x000040a5   Zero   RW          342    .bss                usb_endp.o
    0x200041ed   0x00000003   PAD
    0x200041f0   0x0000001c   Zero   RW          489    .bss                usb_init.o
    0x2000420c   0x000000dc   Zero   RW          574    .bss                rand.o(c_w.l)
    0x200042e8   0x00000060   Zero   RW          664    .bss                libspace.o(c_w.l)
    0x20004348   0x00000000   Zero   RW          467    HEAP                startup_stm32f10x_md.o
    0x20004348   0x00000200   Zero   RW          466    STACK               startup_stm32f10x_md.o


==============================================================================

Image component sizes


      Code (inc. data)   RO Data    RW Data    ZI Data      Debug   Object Name

         0          0          0          0          0         20   core_cm3.o
       392         12          0          0          0      13269   main.o
       224         20          0          0          0     226301   misc.o
      1356         36          0          0          0       2620   qdmx_adc.o
       248         24          0          0          0       1858   qdmx_usb.o
        52         18        236          0        512        484   startup_stm32f10x_md.o
      1058         26          0          0          0      19793   stm32f10x_adc.o
       592         16          0          0          0      13567   stm32f10x_dma.o
      1320         36          0          0          0       7222   stm32f10x_flash.o
       796         18          0          0          0       5163   stm32f10x_gpio.o
       584         38          0          8          0       2630   stm32f10x_it.o
       908         32          0         20          0       8752   stm32f10x_rcc.o
      2904        114          0          4          0       7927   usb_core.o
         0          0        177         26          0        971   usb_desc.o
      1288         82         44         16      16549       2620   usb_endp.o
        60         24          0         20         28       3970   usb_init.o
       820         32          0          4          0       1779   usb_int.o
       140         20          0         62          0       1968   usb_istr.o
        88          6          0          0          0       1326   usb_mem.o
       608         40          0        148          0       7131   usb_prop.o
       352         26          0          7          0       2457   usb_pwr.o
      2088         24          0          0          0      11561   usb_regs.o
       132         12          0          0          0       1418   usb_sil.o

    ----------------------------------------------------------------------
     16012        656        492        320      17092     344807   Object Totals
         0          0         32          0          0          0   (incl. Generated)
         2          0          3          5          3          1   (incl. Padding)

    ----------------------------------------------------------------------

      Code (inc. data)   RO Data    RW Data    ZI Data      Debug   Library Member Name

        90          0          0          0          0          0   __dczerorl2.o
         8          0          0          0          0         68   __main.o
        52          8          0          0          0          0   __scatter.o
        28          0          0          0          0          0   __scatter_zi.o
        12          0          0          0          0         68   exit.o
         6          0          0          0          0        148   heapauxi.o
         6          0          0          0          0          0   libinit.o
         6          0          0          0          0          0   libinit2.o
         2          0          0          0          0          0   libshutdown.o
         2          0          0          0          0          0   libshutdown2.o
         8          4          0          0         96         68   libspace.o
       120         18          0          8        220        116   rand.o
        78          0          0          0          0         76   rt_memclr_w.o
         0          0          0          0          0          0   rtentry.o
        12          0          0          0          0          0   rtentry2.o
         6          0          0          0          0          0   rtentry4.o
         0          0          0          0          0          0   rtexit.o
         8          0          0          0          0          0   rtexit2.o
        20         10          0          0          0         68   sys_exit.o
        74          0          0          0          0         80   sys_stackheap_outer.o
         2          0          0          0          0         68   use_no_semi.o

    ----------------------------------------------------------------------
       548         40          0          8        316        760   Library Totals
         8          0          0          0          0          0   (incl. Padding)

    ----------------------------------------------------------------------

      Code (inc. data)   RO Data    RW Data    ZI Data      Debug   Library Name

       540         40          0          8        316        760   c_w.l

    ----------------------------------------------------------------------
       548         40          0          8        316        760   Library Totals

    ----------------------------------------------------------------------

==============================================================================


      Code (inc. data)   RO Data    RW Data    ZI Data      Debug   

     16560        696        492        328      17408     343068   Grand Totals
     16560        696        492        144      17408     343068   ELF Image Totals (compressed)
     16560        696        492        144          0          0   ROM Totals

==============================================================================

    Total RO  Size (Code + RO Data)                17052 (  16.65kB)
    Total RW  Size (RW Data + ZI Data)             17736 (  17.32kB)
    Total ROM Size (Code + RO Data + RW Data)      17196 (  16.79kB)

==============================================================================

